:1000000000400020115F0000515F0000535F0000BE
:1000100000000000000000000000000000000000E0
:10002000000000000000000000000000555F00001C
:100030000000000000000000575F0000595F000052
:100040005B5F0000054700008D6300005B5F000000
:100050005B5F0000000000005B5F00005B5F000072
:100060005B5F00005D6600005B5F00005B5F00009F
:100070005B5F00005B5F00005B5F00005B5F000098
:100080005B5F0000F56700005B5F00005B5F0000E6
:100090005B5F00005B5F00005B5F00005B5F000078
:1000A0005B5F00005B5F00000000000000000000DC
:1000B0000000000000000000000000000000000040
:1000C00010B5064C2378002B07D1054B002B02D02E
:1000D000044800E000BF0123237010BD4802002047
:1000E00000000000B0CF0000044B10B5002B03D07F
:1000F0000349044800E000BF10BDC04600000000F6
:100100004C020020B0CF0000164B002B00D1144B46
:100110009D46402292029A1A924600218B460F4633
:100120001348144A121A0AF003F90F4B002B00D09F
:1001300098470E4B002B00D0984700200021040068
:100140000D000D48002802D00C4800E000BF0AF066
:10015000AFF82000290006F037F90AF083F8C0460E
:100160000000080000400020000000000000000027
:10017000480200209C2F002000000000000000002A
:100180000123034010D104280CD90268120909D0B8
:10019000531E9B001A1DC1180979002902D0013392
:1001A0009342F8D1180070470023FBE70378002B37
:1001B00003D05AB2002A01DB013070473F2293433B
:1001C000C03B59424B41C01803789343802BF4D174
:1001D0000130F9E710B500240378002B01D120008D
:1001E00010BDFFF7E3FF0134F6E770B5002204000D
:1001F0000D00411C092002F0DBFE002806D001237F
:100200006200134343600023A34200DB70BD9A00E9
:10021000A958821891600133F6E770B5012803DC14
:100220001C2000F091FE70BD01230D6811201D42BD
:10023000F7D04868184206D1042804D90F23026871
:100240001340042B01D00E20EBE702F027FD6D10C8
:100250000400002D03DDFFF7BDFFA84206DA1220DF
:10026000DFE72000FFF7A2FF0400013D012DF8D1D8
:1002700020787F2809DDDF280BDCF8233F22DB0014
:10028000800118406378134018430123400018434D
:10029000C9E7EF280BDCFC22637812019B011340B5
:1002A0003F220007000C0343A0781040ECE7F7283A
:1002B00012DCFC22637892021B031340E0228004CC
:1002C000520310403F221843E3781340FC220343BB
:1002D000A07812018001E8E701204042D5E7F0B59F
:1002E000070085B00D001C20012F06DD4C6801239E
:1002F00022001A40019203D10D2000F025FE54E0A7
:10030000022F02D08A681A42F6D001232E681E42BC
:1003100000D07EE0042E00D87BE01C41002C00DCE5
:100320001C000F2332681340092B29D173685B101E
:100330000193022F05D0AB68019A5B109A4200DD51
:100340000193019B01221F1B0137FB43DB171F4059
:10035000791C092002F02CFE061E09D001237F0023
:100360001F4303002A68083347600199A14202DA5B
:10037000300005B0F0BD0134A100515802C3F4E7CC
:10038000042B46D1300002F089FCFFF723FF0290D6
:10039000022F04D0AB685B10984200DD0293029BF1
:1003A0009C4204DD002002F06FFE0600E0E7300012
:1003B00002F074FC0700019B9C4222DC3000019794
:1003C00002F06CFC03903800FFF7F0FE029B013452
:1003D0000700A342F7DA019BC71A380002F054FE67
:1003E000061EC5D002F05AFC0400286802F056FC34
:1003F000039A019B991A41183A00200009F07CFFEA
:10040000B6E73800FFF7D2FE019B070001330193E6
:10041000D1E7212071E7F8B54D680F00EB0706D44E
:10042000042D04D90F232E683340092B03D00B2051
:1004300000F08AFDF8BD6B6836095C10731EA3429C
:100440000FD80321200007F02FFE6421642803DC6D
:100450000100032800DA03212800891902F0D8FDE1
:1004600005002B6800201B09013B9C42E2D23A6840
:10047000A31C9B005A510123013464001C436C608F
:10048000D8E7F0B585B0012803DC1C2000F05CFD46
:1004900029E001254F682A00022806D08B682B42EC
:1004A00003D05D10002D00DC15000124274200D090
:1004B00074E0042F00D871E00F223B680E681340EF
:1004C000042B25D1264205D1042E03D933681340CD
:1004D000042B01D00E20D9E73800FFF751FEA842C7
:1004E00003DA0120404205B0F0BD380002F0D6FB2F
:1004F0000700300002F0D2FB013D010078190AF03C
:10050000B6FA0028EDD0C01B013040002043EAE7D6
:10051000092B43D17B685B1000939D42E1DC3000E6
:1005200020402ED1042E2BD90F22336820001340F7
:10053000042B26D1300002F0B1FB0F2325000290DE
:100540000393631C01939B00F858864202D1640018
:100550002800DBE728420ED104280CD90368039A4F
:100560001340042B07D102F099FB010002980AF016
:1005700051FA0028EBD0019C009B9C42E1DDB0E7E2
:100580002000431C9A00BA58B24202D14000012414
:10059000BCE71800009B9842F3DDA2E7212075E735
:1005A00010B502F05FFB43000120184310BD0000AE
:1005B00010B57F2902DC0170013010BD1A4B994241
:1005C0000CDC40238A115B42134303703F230B4032
:1005D00080214942194341700230EEE7134B9942A2
:1005E00010DC20230A135B4213433F248022037054
:1005F0008B1152422340214013430A4343708270BF
:100600000330DAE70A4B9942D7DCF0230370603BF2
:100610004370113B8A11FF3B1A4382703F22114005
:100620001943C1700430C8E7FF070000FFFF000056
:10063000FF0F0100F0B50D0085B0002803DC1C2081
:1006400000F082FC0DE009680122080010400AD089
:1006500002AC11412000FFF7ABFF011B200002F0AC
:100660001FFD04001AE004293FD90F230C68234022
:10067000092B3AD14B685B10019303239C46019BE5
:100680009A420EDD02F000FD041E07D02E680125FF
:1006900002F004FB2F00019B9D421DDD200005B0F0
:1006A000F0BD01329300CC580123234001D10D202D
:1006B000C6E764107F2C0DDD0D4E0223B44209DD28
:1006C0000C4E6346B44205DD00270B4EE30FA642F5
:1006D0007B419B00C018D2E70135AB00F15839428D
:1006E000E5D04910FFF764FFD5E72120A8E7C04611
:1006F000FF070000FFFF0000FF0F010010B504001E
:100700000120084010D104290DD90F230A68134095
:10071000042B08D1080002F0C1FA010020000AF001
:1007200079F94342584110BD0020FCE7F7B50F00AE
:10073000012803DC1C2000F007FCFEBD01264D68EB
:100740002E4006D1042D04D90F222B681A40092A05
:1007500001D00B20EFE76A681B095410A34200D8B0
:100760005C1E39681E48FFF7C9FF0123019000286D
:1007700013D139681B48FFF7C1FF002811D0002CA6
:100780000DD00123621C013C9C4092005351234335
:100790006B6004E00136B200AB50B442FADA0020DC
:1007A000CBE73B680D20DA07C5D55B10002B11DDC8
:1007B0009C420FDB9B00A200291DEB188918043313
:1007C000994209D10123013C9C40AA181C43536063
:1007D0006C60E4E71220AEE758681860EFE7C046A7
:1007E0008BB900008FB90000002310B50C000B700E
:1007F000C30705D50D49421020000AF0DDF808E0D6
:100800000B49002802D0042804D10A4920000AF02C
:10081000F3F810BD0428FCD90F2302681340042B01
:10082000F7D102F03BFA04490200E5E7ECC1000011
:1008300094B900009AB900009FB90000F0B593B0D8
:100840000390030002911C20012B1DDD029B01255A
:100850001B681C002C4000D0A8E0042B00D8A5E0A9
:100860001A680F231A40092A48D10194019A029963
:1008700092008A5816002E4005D1042A03D9106828
:100880001840092804D0222000F05EFB07002CE06D
:1008900052685210A418019A013201920199039AE8
:1008A0008A42E3D1611C012202F082FB071E01D1C2
:1008B00000271AE064002543456005000835029AC8
:1008C000B300D1584B680A685B1012099A4200D8ED
:1008D000531E002293420BDCDA43D21713409B00D5
:1008E000ED18019B01369E42E9DB380013B0F0BDE4
:1008F00090000C18A46801322C50EBE7042A55D163
:100900002F0026001D00029AB300D058384237D17C
:10091000042835D903682B40042BB4D1FFF730FCF1
:10092000039B01362418B342EDD1200002F0ACFB4A
:10093000071EBDD0039B029D9B00EB18041D029374
:1009400001232E681E4222D1042E20D90F223368A3
:100950001340042B0DD13000FFF712FC0190300042
:1009600002F09CF9019A0100200009F0C5FC019BEE
:10097000E418029B0435AB42E2D100232370B4E7B4
:1009800005A9FFF731FF05A80AF056F8C8E705A941
:100990003000FFF729FF05A80AF04EF80600020014
:1009A00005A9200009F0A8FCA419E2E7212000F025
:1009B000CBFA7DE7F0B50D0095B0002806DC1C20D1
:1009C00000F0C2FA0400200015B0F0BD0C6801214F
:1009D00023000B40009306D1042C04D922680F3366
:1009E0001A40092A01D00B20EAE7626852100392EC
:1009F000002A03DC009802F047FBE3E73F4A01923C
:100A000001280BD06868084208D1042806D902687A
:100A10001340042B02D102F041F9019001980AF031
:100A20000BF806000F27039B0834013B04935E4339
:100A3000039B02909B001B19059301232068184219
:100A400051D104284FD903683B40042B52D1FFF702
:100A500097FB059B04343618A342EED1300002F018
:100A600013FB041EAFD02B680593029B002B03D011
:100A7000686802F013F90190200002F00FF90500F8
:100A8000009B059A9B00D3189F68380002F006F976
:100A9000012306001F4201D1042F04D807A9380002
:100AA000FFF7A2FE07AE300009F0C6FF0700020004
:100AB0003100280009F020FC029BED19002B0AD020
:100AC000049B009A934206DD2800029A019909F0DE
:100AD00013FC029BED18009B01330093009A039BCB
:100AE0009342CDD16FE707A9FFF77EFE07A809F073
:100AF000A3FFAEE702F0D2F8F9E7C046EEBC000073
:100B000010B50224002806DD0B68DA0703D55C1057
:100B1000022C00DA0224611C0122092002F048FAAA
:100B2000002803D0012364001C43446010BD0B68FF
:100B300070B518000125284032D1042B30D90F247C
:100B40001A6849681440092C16D15C6812092C41B6
:100B5000A24200D8541E844205DC02200132904299
:100B600006DB00200FE085005D19A9600130F2E787
:100B7000840019510130F2E7032C11D1294203D12D
:100B8000132000F0E1F970BD4910FF29F8D81209CF
:100B9000043392009A189A42E3D919700133FAE7A4
:100BA0000B2000F0D1F9DCE70123F7B500264D68F2
:100BB0000F002B400093B3420DD11E00042D0AD923
:100BC0000F222B681A40092A0FD16A681B09561098
:100BD000B34200D85E1E3968CB0713D54C10002CE9
:100BE00001DDA64219DA12202EE0042A04D12800E1
:100BF000FFF7C6FA0600EEE7009E032AEBD11E09B6
:100C0000B600E8E72E48FFF779FD002814D009F078
:100C10006FFE310007F02EFB4C1C009B002B4CD1CB
:100C2000042D4AD92A680F331340092B10D10134FF
:100C3000A40064592000FEBD39682248FFF75EFD1C
:100C400034000028E9D1113000F07EF90400F1E70A
:100C5000042B2AD1280002F021F80600FFF7BAFA87
:100C6000A042C0DB012C1ADC280002F017F800902B
:100C70003000FFF79BFA851B280002F005FA041EDE
:100C8000D8D002F00BF80190786802F007F8009BCA
:100C90002A00F11A4118019809F02EFBCAE730002A
:100CA000FFF784FA013C0600DCE7032B05D12C1981
:100CB000E478023B64001C43BCE70B20C4E7C04659
:100CC00084B900008FB90000F7B54C680F0001200F
:100CD000210001402AD1042C28D90F222368BE68A4
:100CE0001A40092A13D162681B0955100191AB42C1
:100CF00000D85D1E39682848FFF700FD002829D07C
:100D00000F2322681340092B19D1012313E0032A72
:100D10000CD1064203D1132000F016F9FEBD72106B
:100D20000192FF2AF7D81D09AD00E3E70B20F3E796
:100D300001339A00A6509D42FADA0020EEE7032B19
:100D4000FBD1230001331A1BAA42F6DC6A46127952
:100D5000DA70F7E73968CB0706D54910002901DDBD
:100D60008D4209DA1220D7E70C48FFF7C7FC2900AB
:100D7000002801D11130CFE70F2322681340092B3F
:100D800003D1013189000E51D7E7032BD5D16B4632
:100D90001B796418E370D0E78BB900008FB90000AD
:100DA00010B501240868204216D1042814D90F2256
:100DB00003681A40092A01D1406810BD032A03D1F3
:100DC0001809C0002043F8E7042A05D101F066FFA6
:100DD000FFF700FA4000F5E70B2000F0B5F8ECE76C
:100DE00010B5034A0A21034803F084FD10BDC04634
:100DF00034B900002CB9000002000120104001D0DD
:100E0000501070470D22014B1A70FAE7880200203B
:100E1000F0B585B00393019002912C4E2C4B002A23
:100E200002D002223270013A00251A601B68F55484
:100E3000019B9D4201DB05B0F0BD029AAB00D0588A
:100E4000234B1C68C8239B0037191C1B0123184225
:100E500006D0204A43102100380009F07BFD09E04C
:100E60001D4A002802D004281BD11C4A210038004A
:100E700009F070FD300009F0DFFD154A039B10609A
:100E8000002B0CD0019B013BAB4208DD144B984278
:100E900005D8431C1360202232540022F25401353D
:100EA000C6E704280FD90F2302681340042B04D18E
:100EB00001F0F4FE0B4A0300CDE7092B04D143688F
:100EC000094A5B10C7E70123084AC4E789020020EA
:100ED000AC050020ECC1000094B900009AB90000F4
:100EE0001F030000E3C7000004BC000013BC0000A7
:100EF0000123020010B51A4015D1042801D9026857
:100F000012090B4011D1042901D90B681B090024D7
:100F1000934206D104309B000431C318984206D393
:100F20000124200010BD0022EBE70023EFE7047846
:100F30000A78002C01D1002AF2D00130013194420C
:100F4000ECD00024EDE70000014B18700020704742
:100F50008802002070B501F0B5FC094C0100251D88
:100F60001F22280009F06FFD280009F065FD042309
:100F700004308008000118432060200070BDC04686
:100F800064020020C368F0B59D00836889B05D19D4
:100F90000300183306930369069A9F00069B02908C
:100FA000DF19436901939B00D3180393CD4B1B7842
:100FB000002B26D17F222B68CB491C1213409B00AB
:100FC0005B58043501929F46029B587804F066F8FE
:100FD0000023029A137027E0C24B1B78002B10D11C
:100FE0002B68019A1C121340BF4A9B009B58043582
:100FF000E9E7069B3A1DD11ABA4BD82928DD1A22F7
:101000001A70029BB74C9B6821780193EA1A029BE5
:1010100092109B7812021A43029B587804F046F80B
:101020000023029A23701370029B069A9B68019317
:10103000ED1A029BAD10DD60069BFE1A029BB610F6
:101040001E61039B9B1A029A9B10536109B0F0BD6D
:101050001B783C60002B01D01700D2E72B68019968
:101060001C120B40A0499B005B5817000435AAE7EF
:10107000069B3A1DD11A9B4BD82902DD1A221A7001
:10108000BFE728681B78291D3860002B02D01700A5
:101090000D00B6E76B6801991C120B4092499B004A
:1010A0005B58170008358EE7069B3A1DD11A8D4B09
:1010B000D82902DD1A221A70A3E7A4001B782C1984
:1010C0003C60002B01D017009BE72B6801991C1294
:1010D0000B4085499B005B581700043573E7069B5E
:1010E0003A1DD11A7F4BD82902DD1A221A7088E7DF
:1010F0007E49A40061581B783960002B01D017008D
:101100007FE72B6801991C120B4077499B005B58C5
:101110001700043557E7043F744B3A68A400E250C7
:10112000704B1B78002B00D06BE72B68019A1C12C8
:1011300013406D4A9B009B58043544E76B4BA40059
:10114000E058FFF759FE043F06003868FFF754FEE9
:1011500036180120654B76000643E650614B1B783C
:10116000002B00D04DE72B68019A1C1213405E4AF9
:101170009B009B58043526E7069B3A1DD11A594B14
:10118000D82902DD1A221A703BE70698039C012138
:10119000A04202D221000C3909681B783960002B6B
:1011A00001D017002DE72B6801991C120B404E4906
:1011B0009B005B581700043505E7069B3A1DD11AC2
:1011C000484BD82902DD1A221A701AE706990398AB
:1011D00081420FD203000C3B1B6845495B10641829
:1011E000E41AA40023583B603E4B1B78002B05D02B
:1011F000170006E7182119700023F4E72B680199FE
:101200001C120B4038499B005B5817000435DAE686
:10121000069B039A934219D213000C3B1B68344A75
:10122000043FA4185B10E31A039A39689B00995095
:101230002C4B1B78002B00D0E3E62B68019A1C1284
:101240001340294A9B009B580435BCE61822254BC5
:101250001A70EDE7069B039A93422DD2244B3E1F52
:10126000E31814000C3C04932368049A5B10D31A0F
:10127000039A9B009858FFF7BFFD07903068FFF76F
:10128000BBFD2468049B64101C1B079BA4001F1853
:1012900001207F00039B0743E7503700114B1B7869
:1012A000002B00D0ADE62B68019A1C1213400E4AA9
:1012B0009B009B58043586E618220A4B1A70EDE70E
:1012C000069B3A1DD11A074BD82902DD1A221A7043
:1012D00097E60399A40061581B783960002B09D068
:1012E00017008EE68802002004BA0000442D00207A
:1012F000FDFFFF3F2B6801991C120B40D7499B0053
:101300005B58170004355EE6043F039B3A68A4006F
:10131000E250D34B1B78002B00D072E62B68019A69
:101320001C121340CD4A9B009B5804354BE6039B8F
:10133000A4001C192368043F38685E10FFF75CFDA9
:1013400036180120C64B76001B7806432660002B1A
:1013500000D056E62B68019A1C121340BF4A9B002E
:101360009B5804352FE6069BA4003F1BBC4CBB4298
:101370000CD82378002B00D043E62B68019A1C126E
:101380001340B64A9B009B5804351CE6B54801F053
:1013900075FC2378002B00D033E62B68019A1C12D1
:1013A0001340AE4A9B009B5804350CE6A300ED1891
:1013B000002C00DA38E6AA4B1B78002B00D020E680
:1013C0002B68019A1C121340A44A9B009B580435B9
:1013D000F9E5043F3B68042B04D1A300ED18002C71
:1013E00000DA21E69E4B1B78002B00D009E62B6823
:1013F000019A1C121340994A9B009B580435E2E560
:10140000043F3B68042B06D0A200AD18002C02DA82
:10141000002B00D108E6924B1B78002B00D0F0E5A2
:101420002B68019A1C1213408C4A9B009B58043570
:10143000C9E53A1F13685B10013B002B06DD012153
:101440005B00A4000B432D191360EDE5844B1700DE
:101450001B78002B00D0D4E52B68019A1C12134096
:101460007E4A9B009B580435ADE53A00069B0C3242
:10147000D31AD82B03DD1A22794B1A70C1E5FF234A
:1014800061005B001940FE3BFF3B19433960029944
:1014900006988968241204916D1A0299AD10897812
:1014A0002D020D4303999D40091A891099401D434F
:1014B0000B43BB60029B7D609C70E4B26A4BE4000E
:1014C0000392E358029A9360654A1278002A03D087
:1014D00008331D00039F94E51D00019A9B680C359D
:1014E0001C1213405D4A9B009B58039F6BE53B1FFA
:1014F0001C68039A069B93422DD10A20E3070CD463
:10150000042C13D90F2322681340042B11D120007F
:1015100001F0C4FB09F090FA0630643003F07AFA67
:1015200000280FD1043D069B03937DE50720042C82
:10153000F3D02000431E9841FA234042FF33184065
:101540000730EAE7029B2100587803F0C1FD002331
:10155000029A1370E7E7039B039A0C3B1B680299FE
:101560005B109B00D31A0C3B1C601F1D1300083B33
:101570001B685A108A70D2B23B49D2005B005558A2
:101580009B0A029A9B009560ED18039B069A043B08
:101590001B685B109B00D3180393314B1B78002B07
:1015A00000D02EE52B68019A1C1213402B4A9B0099
:1015B0009B58043507E53B1F1868FFF71DFCA40086
:1015C00006003F1B1E2827DC00280DDC244B1B785F
:1015D000002B00D015E52B68019A1C1213401F4AFE
:1015E0009B009B580435EEE401F05AF9033E36188F
:1015F00001F056F91D4B801B9842F9D8184B1B7807
:10160000002B00D0FDE42B68019A1C121340134AF2
:101610009B009B580435D6E40123029A137001F015
:101620003FF9029B0A3886195E60FDE43B1F18688B
:10163000FFF7E2FBA40006003F1B002818DC084B64
:101640001B78002B00D0DCE42B68019A1C1213409D
:10165000024A9B009B580435B5E4C04604BA00001A
:101660008802002025BC00004C2500209F86010038
:10167000CD4B984203DD1D22CC4B1A70C1E40123EF
:10168000029A137001F00CF9FA239B005E43029B4F
:101690000A3E30185860C7E4A300FF1A0023200058
:1016A0001A003900FFF7B4FBC14EC24C316820006C
:1016B00003F0C6FB3168200003F011FD3168200003
:1016C00001F08AFDB94B1B78002B00D099E42B6800
:1016D000019A1C121340B84A9B009B58043572E4CF
:1016E000B24BA4001B783F1B002B00D089E42B6871
:1016F000019A1C121340B04A9B009B58043562E4C7
:10170000029803F0EBF9A94B1B78002B00D078E48A
:101710002B68019A1C121340A74A9B009B58043562
:1017200051E43B1F1B68002B3DD13B000C3B1B6869
:10173000DA072BD5390001225B1058000839024323
:101740000A60002B43DD012259001143381F01605C
:101750003900083909681141CB1A39000C39096878
:10176000114223D09B189340A4001343039AA35023
:101770008E4B1B78002B00D043E42B68019A1C127F
:1017800013408D4A9B009B5804351CE4042B06D95A
:101790000F2219680A40092A01D15B68CAE7192299
:1017A000824B1A702DE45B10013BCAE7042909D96A
:1017B0000F2208680240092A04D102339B005B58BB
:1017C000A400D3E71922794B1A70FFF71AFC0435ED
:1017D000CEE7A300069AFB189B1AD82B13DC012234
:1017E000631E002C14DC714B1B78002B01D0FFF71B
:1017F00008FC2B68019A1C1213406F4A9B009B58EF
:101800000435FFF7E0FB1A22684B1A70FFF7F9FB6B
:101810003A601C000437E3E7069A3B1D9B1A634EAF
:10182000D82B03DD1A233370FFF7EBFB069B039ADB
:10183000A40093422AD23B1F1868FFF7DDFA011E6D
:1018400021DD039B0C3B1A68521082421BDB900780
:10185000801A5A4B4018C018039B8000C2583B1B8B
:101860001A60524B3F1B1B780437002B01D0FFF747
:10187000C8FB2B68019A1C1213404F4A9B009B58CF
:101880000435FFF7A0FB20233370EAE71823FBE7BA
:10189000A3009C46FE1A002C17DC1C22434B1A7036
:1018A000002333606346FF1A404B04371B78002B3C
:1018B00001D0FFF7A6FB2B68019A1C1213403E4A89
:1018C0009B009B580435FFF77EFB002033685A10BD
:1018D0008300F15801230B4003D10D21334A1170CD
:1018E000DFE749108A4200DD0A0001308442EFDC64
:1018F000012352001343D4E7A3009C46FE1A002C98
:1019000017DC1C22294B1A70002333606346FF1A30
:10191000264B04371B78002B01D0FFF772FB2B6896
:10192000019A1C121340244A9B009B580435FFF770
:101930004AFB002033685A108300F15801230B4002
:1019400003D10D21194A1170DFE749108A4200DAEC
:101950000A0001308442EFDC012352001343D4E734
:101960003B00083B1868FFF747FA3B1F0600186862
:10197000FFF742FA0023864200DA0433A4003A1B40
:1019800017001360094B04371B78002B01D0FFF7B9
:1019900038FB2B68019A1C121340074A9B009B5886
:1019A0000435FFF710FBC04680EE360088020020A9
:1019B000AC0500208902002004BA0000FCFFFF3FB4
:1019C0003B00083B1868FFF717FA3B1F0600186832
:1019D000FFF712FAF30FC217B0425341A4003A1BAB
:1019E00017009B001360E14B04371B78002B01D0DC
:1019F000FFF707FB2B68019A1C121340DC4A9B007F
:101A00009B580435FFF7DFFA3B00083B18683B1F83
:101A10001968A600BE1B0423814202D0042802D804
:101A20000023336016E001231842F9D10F23026826
:101A30001A40042AF4D1033A1142F1D10429EFD912
:101A40000A681340042BEBD1FFF752FA431E98416A
:101A500080003060C54BA4001B783F1B0437002B6F
:101A600001D0FFF7CEFA2B68019A1C121340C04A2E
:101A70009B009B580435FFF7A6FA3B00083B18680B
:101A80003B1F1968A600BE1B0023814202D0042818
:101A900002D80423336016E001231842F9D10F2342
:101AA00002681A40042AF4D1033A1142F1D1042900
:101AB000EFD90A681340042BEBD1FFF719FA434220
:101AC000584180003060A94BA4001B783F1B0437AD
:101AD000002B01D0FFF795FA2B68019A1C121340D6
:101AE000A34A9B009B580435FFF76DFA3B00083B67
:101AF0001868FFF781F93B1F06001868FFF77CF9AB
:101B0000F317C20F86425341A4003A1B17009B00F3
:101B10001360964B04371B78002B01D0FFF771FA46
:101B20002B68019A1C121340914A9B009B58043564
:101B3000FFF749FA3B00083B1868FFF75DF93B1FC8
:101B400006001868FFF758F90023864200DD0433C9
:101B5000A4003A1B17001360844B04371B78002B3A
:101B600001D0FFF74EFA2B68019A1C121340804AED
:101B70009B009B580435FFF726FA3B1F1B68A40007
:101B8000043B5A1E93413A1B17009B001360774B8E
:101B900004371B78002B01D0FFF733FA2B68019A2A
:101BA0001C121340724A9B009B580435FFF70BFA36
:101BB0003B00083B1868FFF71FF93B1F0600186839
:101BC000FFF71AF932180120A4003B1B1F00520036
:101BD00002431A60654B04371B78002B01D0FFF7D6
:101BE00010FA2B68019A1C121340614A9B009B5803
:101BF0000435FFF7E8F93B00083B1868FFF7FCF8ED
:101C00003B1F06001868FFF7F7F8321A0120A400FE
:101C10003B1B1F00520002431A60544B04371B78D1
:101C2000002B01D0FFF7EDF92B68019A1C1213402D
:101C30004F4A9B009B580435FFF7C5F93B00083B12
:101C40001868FFF7D9F83B1F06001868FFF7D4F8AB
:101C500002000120A4003B1B1F00724352000243FC
:101C60001A60424B04371B78002B01D0FFF7C9F9EB
:101C70002B68019A1C1213403D4A9B009B58043567
:101C8000FFF7A1F93B1F1868FFF7B6F8061E17D13A
:101C90001F22364B1A70A4003B1B1F001E60334BE3
:101CA00004371B78002B01D0FFF7ABF92B68019AA2
:101CB0001C1213402E4A9B009B580435FFF783F9F2
:101CC0003B00083B1868FFF797F8310006F0ECF985
:101CD000012640000643DEE73B1F1868FFF78CF83B
:101CE000061E17D11F22214B1A70A4003B1B1F0098
:101CF0001E601E4B04371B78002B01D0FFF781F9C3
:101D00002B68019A1C121340194A9B009B580435FA
:101D1000FFF759F93B00083B1868FFF76DF83100F1
:101D200006F0A8FA012649000E43DEE73B1F1868BB
:101D3000FFF762F8C217801850400122A4003B1B35
:101D40001F00400010431860084B04371B78002B1D
:101D500001D0FFF756F92B68019A1C121340044A70
:101D60009B009B580435FFF72EF9C04688020020DF
:101D700004BA0000A300FE1A3068012C24D1FFF73A
:101D80003BF80494079008F0B3FD0799002900DCA4
:101D9000012106F06FFA049BA400C9180123490031
:101DA0001943F34B3F1B1B7831600437002B01D0E4
:101DB000FFF727F92B68019A1C121340ED4A9B008C
:101DC0009B580435FFF7FFF8FFF716F8049070688A
:101DD000FFF712F8049B0130C31A0793D3E7A3005F
:101DE000FE1A31002000049301F096F9049B306044
:101DF000FF1ADF4B04371B78002B01D0FFF701F9E6
:101E00002B68019A1C121340DA4A9B009B58043538
:101E1000FFF7D9F83B00083B1868FEF7EDFF3B1FC2
:101E200006001868FEF7E8FF02000120A4003B1B33
:101E30001F003240520002431A60CD4B04371B781A
:101E4000002B01D0FFF7DDF82B68019A1C1213401C
:101E5000C84A9B009B580435FFF7B5F83B00083B88
:101E60001868FEF7C9FF06003B1F1868FEF7C4FF9D
:101E7000320002430120A4003B1B1F00520002431A
:101E80001A60BB4B04371B78002B01D0FFF7B9F861
:101E90002B68019A1C121340B64A9B009B580435CC
:101EA000FFF791F83B00083B1868FEF7A5FF060016
:101EB0003B1F1868FEF7A0FF320042400120A4003B
:101EC0003B1B1F00520002431A60A94B04371B78CA
:101ED000002B01D0FFF795F82B68019A1C121340D4
:101EE000A44A9B009B580435FFF76DF83B1F186808
:101EF000FEF782FFC0430122A4003B1B1F004000ED
:101F0000104318609A4B04371B78002B01D0FFF761
:101F100078F82B68019A1C121340964A9B009B5834
:101F20000435FFF750F83B00083B1868FEF764FFE4
:101F300006003B1F1868FEF75FFF32008240510029
:101F40000122A4003B1B1F000A431A60884B043780
:101F50001B78002B01D0FFF754F82B68019A1C1254
:101F60001340844A9B009B580435FFF72CF83B0034
:101F7000083B1868FEF740FF06003B1F1868FEF795
:101F80003BFF3200024151000122A4003B1B1F0015
:101F90000A431A60764B04371B78002B01D0FFF7F9
:101FA00030F82B68019A1C121340724A9B009B5810
:101FB0000435FFF708F83B000C3B1868FEF71CFFE0
:101FC0003B00083B06001868FEF716FFF1170200F9
:101FD000C317300006F0A0F93B1F04900591186864
:101FE000FEF70AFF02000498059906F049F943003C
:101FF0000120A4003E1B370018435D4B30601B7866
:102000000437002B01D0FEF7FCFF2B68019A1C124D
:102010001340584A9B009B580435FEF7D4FFA30099
:10202000FE1A310020000493FEF76AFD049B306025
:10203000FF1A4F4B04371B78002B01D0FEF7E1FF4E
:102040002B68019A1C1213404A4A9B009B58043586
:10205000FEF7B9FFA300FF1A39002000FEF767FD65
:10206000434B1B78002B01D0FEF7CBFF2B68019A66
:102070001C1213403F4A9B009B580435FEF7A3FFF8
:10208000A300FE1A310020000493FEF78DFD049B8F
:102090003060FF1A364B04371B78002B01D0FEF757
:1020A000B0FF2B68019A1C121340324A9B009B58C8
:1020B0000435FEF788FFA300FF1A39002000FEF761
:1020C00003FE2B4B1B78002B01D0FEF79AFF2B68E9
:1020D000019A1C121340274A9B009B580435FEF7B7
:1020E00072FFA300FE1A310020000493FEF758FE91
:1020F000049B3060FF1A1E4B04371B78002B01D065
:10210000FEF77FFF2B68019A1C121340194A9B00AF
:102110009B580435FEF757FF069B3E1DF31A144CDF
:10212000D82B03DD1A232370FEF76BFF00F0C2FBF0
:1021300043000120184323783860002B02D0370079
:10214000FEF75FFF2B68019A1C121340094A9B009F
:102150009B5837000435FEF736FF069B3E1DF31AE9
:10216000034CD82B08DD1A232370FEF74AFFC04624
:102170008802002004BA000000F092FBF54B4000FA
:1021800018400123184323783860002B02D0370011
:10219000FEF737FF2B68019A1C121340EE4A9B0092
:1021A0009B5837000435FEF70EFF0123A600BE1B27
:1021B00020001A003100FEF72BFEE84C2068643046
:1021C00002F028FC002802D1043DFEF72DFF029BFF
:1021D00021685A78E24802F090FF0123029A370002
:1021E000137000F05DFBDF4B22681B68063253431F
:1021F0001818029B5860FEF717FFA600BE1B2000B0
:10220000012300223100FEF703FED44C2068643025
:1022100002F000FC0028D7D0D14802F069FDDCE7CD
:10222000A4003E1BFEF796FE3700CF4B30601B78B4
:102230000437002B01D0FEF7E4FE2B68019A1C1234
:102240001340C54A9B009B580435FEF7BCFEA40012
:102250003E1B300000F05DFB3700C34B30601B7845
:102260000437002B01D0FEF7CCFE2B68019A1C121C
:102270001340B94A9B009B580435FEF7A4FEA40006
:102280003E1B300000F047FB3700B74B30601B7837
:102290000437002B01D0FEF7B4FE2B68019A1C1204
:1022A0001340AD4A9B009B580435FEF78CFEA300FB
:1022B000FE1A31002000049300F030FB049B3060D4
:1022C000FF1AA94B04371B78002B01D0FEF799FEAB
:1022D0002B68019A1C1213409F4A9B009B5804359F
:1022E000FEF771FEA4003F1B380000F049FB9E4B37
:1022F0001B78002B01D0FEF784FE2B68019A1C127C
:102300001340954A9B009B580435FEF75CFEA300E2
:10231000FE1A31002000049300F05AFB049B306049
:10232000FF1A914B04371B78002B01D0FEF769FE92
:102330002B68019A1C121340874A9B009B58043556
:10234000FEF741FEA4003F1B380000F083FB864BE4
:102350001B78002B01D0FEF754FE2B68019A1C124B
:1023600013407D4A9B009B580435FEF72CFE01214B
:10237000200000F057FB7C4B1B78002B01D0FEF7B0
:1023800040FE2B68019A1C121340734A9B009B5815
:102390000435FEF718FE0021200000F043FB724BCD
:1023A0001B78002B01D0FEF72CFE2B68019A1C1223
:1023B0001340694A9B009B580435FEF704FEA400B5
:1023C0003E1B300000F068FB3700674B30601B7825
:1023D0000437002B01D0FEF714FE2B68019A1C1263
:1023E00013405D4A9B009B580435FEF7ECFDA400AA
:1023F0003E1B300000F064FB37005B4B30601B7805
:102400000437002B01D0FEF7FCFD2B68019A1C124B
:102410001340514A9B009B580435FEF7D4FDA4009D
:102420003F1B380000F026FB4F4B1B78002B01D0E0
:10243000FEF7E7FD2B68019A1C121340464A9B00E9
:102440009B580435FEF7BFFDA4003F1B380003F086
:1024500001F9454B1B78002B01D0FEF7D2FD2B680C
:10246000019A1C1213403C4A9B009B580435FEF70E
:10247000AAFDA4003E1B300003F094F937003A4B4C
:1024800030601B780437002B01D0FEF7BAFD2B68B3
:10249000019A1C121340304A9B009B580435FEF7EA
:1024A00092FDA4003F1B380003F0A4F82E4B1B78CC
:1024B000002B01D0FEF7A5FD2B68019A1C121340DA
:1024C000254A9B009B580435FEF77DFDA4003E1B6A
:1024D000300003F0A5F83700234B30601B78043739
:1024E000002B01D0FEF78DFD2B68019A1C121340C2
:1024F000194A9B009B580435FEF765FDA300FF1A9F
:102500003900200001F010F9174B1B78002B01D087
:10251000FEF777FD2B68019A1C1213400E4A9B00B0
:102520009B580435FEF74FFDA300FF1A3900200029
:1025300000F082FF0C4B1B78002B01D0FEF761FDF1
:102540002B68019A1C121340034A9B009B580435C8
:10255000FEF739FDFEFFFF7F04BA0000AC05002046
:10256000890200200400002088020020A300FF1A36
:102570003900200000F070FF944B1B78002B01D035
:10258000FEF73FFD2B68019A1C121340904A9B00F6
:102590009B580435FEF717FDA300FF1A39002000F1
:1025A00000F082FF894B1B78002B01D0FEF729FD3C
:1025B0002B68019A1C121340854A9B009B580435D6
:1025C000FEF701FDA300FE1A31002000049303F082
:1025D00064F9049B3060FF1A7C4B04371B78002B96
:1025E00001D0FEF70EFD2B68019A1C121340784AA9
:1025F0009B009B580435FEF7E6FCA300FE1A310051
:102600002000049303F051F9049B3060FF1A6F4BD4
:1026100004371B78002B01D0FEF7F3FC2B68019ADE
:102620001C1213406A4A9B009B580435FEF7CBFCF2
:10263000A300FE1A31002000049303F03EF9049B2E
:102640003060FF1A614B04371B78002B01D0FEF776
:10265000D8FC2B68019A1C1213405D4A9B009B58C2
:102660000435FEF7B0FCA300FE1A310020000493ED
:1026700003F02BF9049B3060FF1A544B04371B788E
:10268000002B01D0FEF7BDFC2B68019A1C121340F1
:102690004F4A9B009B580435FEF795FCA300FF1A98
:1026A0003900200000F0C8FF484B1B78002B01D0F8
:1026B000FEF7A7FC2B68019A1C121340444A9B00AA
:1026C0009B580435FEF77FFCA300FF1A3900200059
:1026D00000F012FF3D4B1B78002B01D0FEF791FC60
:1026E0002B68019A1C121340394A9B009B580435F1
:1026F000FEF769FCA300FE1A31002000049300F0ED
:1027000069FE049B3060FF1A304B04371B78002BA6
:1027100001D0FEF776FC2B68019A1C1213402C4A5C
:102720009B009B580435FEF74EFCA300FF1A3900AE
:10273000200000F0DFFF254B1B78002B01D0FEF7B7
:1027400060FC2B68019A1C121340214A9B009B5885
:102750000435FEF738FC069B029AFB1A9B101361A6
:10276000A300FF1A3900200002F0D8F8174B1B789D
:10277000002B01D0FEF745FC2B68019A1C12134078
:10278000134A9B009B580435FEF71DFC069B029ADA
:10279000FB1A9B101361A300FE1A31002000049362
:1027A00002F0BCF8049B3060FF1A084B04371B781A
:1027B000002B01D0FEF725FC2B68019A1C12134058
:1027C000034A9B009B580435FEF7FDFB880200205E
:1027D00004BA00000023F7B55A1E0192002B07DA55
:1027E00000F0B8FF02F086FB02F0DEFC1923019333
:1027F00000263000194B1968B14212DD184B1A68D7
:1028000001328A420FDAF0241A601D68154F6C43BA
:10281000E35D002B1FD0E419022B06D12000FEF748
:10282000B1FB019BD8E70022EDE7012B0DD1002879
:1028300001D100F035F8F0226A43BB185B680A4901
:10284000C31A8B4201D80223BB54F0235D43054BCE
:10285000EB5C022BE2D00136CCE7C046B00500208D
:1028600000000020EC1B00209F8601000020704724
:102870000020704700207047002070470122002090
:10288000054B06491A61585004310330585008313D
:10289000801858501A6070470080004004050000FE
:1028A0000122034B1A64A822D20098587047C046F0
:1028B0000080004010B5FFF7F3FFFA21890005F012
:1028C00069FB10BD0048704778BC00001A207047B3
:1028D00070B5054E0400335C0D008B4202D003F04E
:1028E00009FF355570BDC046B405002070B5002401
:1028F000064D635D012B05D10021200003F0FAFE97
:102900000023635501341A2CF2D170BDB4050020A8
:1029100070470D207047352070470000F8B501243E
:102920000B6806000D00234204D10D20FEF70CFBBE
:102930002000F8BD5B102000052BFAD80E4A9B0042
:102940009C580E4F3B5D002B05D00021200003F06A
:10295000D1FE00233B55012E06DD6B68042B03D10D
:102960000221200003F0C6FE200003F071FD0124C7
:1029700040002043DDE7C04660BC0000B4050020F5
:10298000F8B501260568354202D04468344203D1C7
:102990000D20FEF7D9FAF8BD6D10192DFBD80A4F9E
:1029A0007B5D012B04D03100280003F0A3FE7E558F
:1029B000064964108C4202DCE143C917214028001B
:1029C00003F0CCFDE7E7C046B4050020FF0300009C
:1029D00070B501240D68254204D10D20FEF7B4FA2C
:1029E000200070BD6D10192D17D80024012804DDBA
:1029F0004C68043C63425C416400094E735DA34231
:102A000004D02100280003F075FE7455280003F05F
:102A1000A5FE03000420012BE3D00020E1E7C0461F
:102A2000B405002070B504000D0019280ED8084E1A
:102A3000335C012B04D0012103F05CFE01233355EC
:102A4000290020004D1EA94103F072FE70BDC04652
:102A5000B4050020036810B5DA0703D40D20FEF793
:102A600073FA10BD4168581004394A425141FFF7CA
:102A7000D9FFF6E737B569460A00064B30CB30C2BE
:102A800003680220042B02D100F0E6FC37BD00F001
:102A90000BFDFBE738BC000010B5084C237D002B74
:102AA00005D00021142003F025FE002323751420F7
:102AB00003F054FE43425841800010BDB40500208D
:102AC00010B5084CA37D002B05D00021162003F083
:102AD00011FE0023A375162003F040FE4342584127
:102AE000800010BDB40500207047704710B5034A40
:102AF0000421034801F0FEFE10BDC04640BC0000AA
:102B00001CC30000E12170B54902144803F098FA93
:102B1000FFF7B4FE0A2003F095FC0023FF21104AC2
:102B2000995401331A2BFBD1012200200D4B0100D7
:102B30001A6004230C4A0D4D1468002CFCD02C683C
:102B40000002013B20431160002BF5D10122084B0C
:102B50001A6003F031FC00F049FF70BD741B0020C7
:102B6000B405002000D0004000D1004008D500404E
:102B700004D00040F8B50B4E070030000D0003F004
:102B8000A7FA0400A84200DD2C003D00EB1B9C428C
:102B900005DD300003F0A6FA28700135F6E72000C5
:102BA000F8BDC046741B002010B50100014803F0B9
:102BB0004FFA10BD741B002010B5054C200003F027
:102BC00055FAE1212000490203F03AFA10BDC0464F
:102BD000741B0020C3070CD4064B1B68834208D823
:102BE000054B1B68984204D8031F1B68002B00D0BC
:102BF00018007047D8050020D405002000230120CC
:102C000010B509499A0001338850642BFAD1074C5A
:102C1000074A0021200007F08BFB064B064A636041
:102C2000064B1A6010BDC046442D0020DC05002074
:102C3000D409000030270000E0050020D005002066
:102C400010B5044B044A1A60044B054A1A60FFF79A
:102C5000D5FF10BDD8050020DC050020D4050020DC
:102C6000B00F0020044B1B68186800090238C343EA
:102C7000DB1718407047C046D005002000B59BB058
:102C80000200054901A807F097FE01A802F04CF8E0
:102C900002F08AFAFCE7C046DEBC00000A4BC2071D
:102CA00004D4042804D8094B00D0094B18007047FD
:102CB0000F2203681A40031D042AF7D0054B092A86
:102CC000F4D0054BF2E7C046C4BC00009AB900003E
:102CD00094B90000D7BC0000CEBC00000020064A1A
:102CE0000649131F186013681B0902339B00D21892
:102CF0008A42F6D37047C046E0050020B00F00209E
:102D0000F7B50F2401262E4B2E4A19682E4B2F4D56
:102D1000186813681F002740072F20D813681B0965
:102D200002339B00D218AA42F3D30024284EA500F8
:102D3000AD192868FFF74EFF01342860642CF6D1E6
:102D4000244C2068002802D0FFF744FF20600025B3
:102D5000214B1B680093009B9D4213DBF7BD1B09B1
:102D60009B00D3189A42D9D01F68374208D1B94284
:102D700006D2B84204D3043F3F68002F00D01F6042
:102D8000043BEFE7F0236B43144A9B181A78002AA0
:102D900001D10135DFE71F693C2300266B43DB19B6
:102DA0009B0001930136BB1BF3D4019BB4001C1B99
:102DB0000A4B1C19A069FFF70DFFA061F2E7C0469E
:102DC000D8050020E0050020D4050020B00F002029
:102DD000442D0020B00F0020B0050020EC1B002087
:102DE000F7B50124204244D1224B1B689C469842EF
:102DF0003FD3214B1B68019398423AD8031F1B68AD
:102E0000002B36D10200036800941B09002B0FD160
:102E10000099131F196090422BD015682B1F1B6857
:102E2000990069180C68013B14600A602A00EDE7FC
:102E30009D0055192968009C214218D18C4516D84F
:102E4000019C8C4213D30E1F3468002C0FD10F68E5
:102E50000F343C40072C07D92F60151F2B600B68DF
:102E60000A601B090A00D1E700993160CEE7013BF7
:102E7000CCE7F7BDD8050020D40500200D49F0B5FA
:102E80000B000F260C4D18681C1F27680209023220
:102E9000002F0BD000208B4200D008002060900053
:102EA000091892009B18AB42EDD3F0BDB0431860F7
:102EB000F7E7C046E0050020B00F0020F8B5114C40
:102EC00026000F2233681F0913420DD07D1CAD0070
:102ED000A64204D02A003100200007F016FA002292
:102EE0006319043564191A600237BF00064BF619DE
:102EF0009E42E6D31B1B9B10013B1B012360034B2F
:102F00001C60F8BDE0050020B00F0020D0050020B7
:102F1000F0B59BB0FFF7C4FC002407001E4AA300D5
:102F2000D0580134FFF75CFF642CF7D11B4B1868B5
:102F3000002801D0FFF754FF0026194B1B689E4262
:102F400016DBFFF79BFFFFF7DBFEFFF7B7FFFFF78F
:102F5000A7FC144BC21B1B6813491B6801A81B0963
:102F6000023B07F029FD01A801F0DEFE1BB0F0BD19
:102F7000F02575430D4BED182B78002B01D1013650
:102F8000DBE72B695C1E002CF9DBA300EB189869CA
:102F9000FFF726FF013CF6E7442D0020B00F00208C
:102FA000B0050020D0050020A4BC0000EC1B0020D0
:102FB000F7B5164D4F1C2B6806001B680C000192DC
:102FC0001B099F420ADBFFF7A3FF2B681B681B0945
:102FD0009F4203DB0A20FDF7B7FFFEBD2868A71C50
:102FE000BA00DB1B81181B010B6029600021031F45
:102FF00019600F231E4003002401264340C3083AF2
:103000009A189A42E9D9019902C3FAE7D00500203B
:10301000F7B503000122134004000D000193002BBB
:103020002AD1164B1B68834226D8154B1B68834256
:1030300022D90F23134F386000681840FFF7B8FFFC
:10304000019B3C68061E3B6016D0236804301B09B8
:103050009D4200DD1D00AA00211D251F07F04CF92F
:10306000FFF73CFE2E60FFF74BFE00232B6022682B
:103070000F339A43226034002000FEBDD8050020A3
:10308000D4050020B00F00200323043010B5C11771
:1030900019400918891000220420FFF789FF10BD8C
:1030A00070B5050008000C00FFF7EEFF00230028B4
:1030B00004D170BDE95CC21811710133A342F9DB80
:1030C000E343DB171C40002304192371F1E70000E0
:1030D00010B501240B681C4016D05C10200005F0D0
:1030E00077FA0B4905F042F907F028F803F07AFC6B
:1030F0000022084B06F0DCF903F01CFC06F0AEFFE2
:1031000043000120184310BD0D20FDF71DFFE5E72A
:10311000D30237390000D040086870B5012405009B
:10312000254006D1042804D90F2302681340042B3C
:1031300003D00E20FDF708FF70BDFFF7AFFD037849
:103140002900233B5A4253411022C01807F02AFDA0
:1031500080239B05C218044B9A4201D91420E9E749
:1031600040002043E8E7C046FFFFFF3F10B5034A99
:103170000221034801F0BEFB10BDC046F4BC0000B4
:10318000EFBC00000020704710B51E20FDF7DCFEEC
:1031900010BD10B51E20FDF7D7FE10BD10B51E20C6
:1031A000FDF7D2FE10BD10B51E20FDF7CDFE10BDFF
:1031B00010B51E20FDF7C8FE10BD10B51E20FDF78E
:1031C000C3FE10BD10B51E20FDF7BEFE10BD10B52C
:1031D0001E20FDF7B9FE10BD7047000010B5034A70
:1031E0000921034801F086FB10BDC04614BD000054
:1031F0005CBD00000120034B1860034B1B6883403B
:1032000018437047D40F0020B40F0020F0B5EFF33F
:1032100010810123194083F31088134C134AA446EC
:103220001268134E013A9340124F134A002B17D0E5
:10323000146803420FD03D682C60C046C046C046AB
:10324000C046C046C046C046C0460C4C15682468FF
:1032500025605B08EAE765462C6014683460F8E78F
:1032600081F31088F0BDC04608050050080000201A
:103270000C050050C00F0020C80F0020BC0F00201C
:1032800030B585B001AD0C220649280007F034F8AE
:103290000024285D01210134FFF71AFB0C2CF8D122
:1032A00005B030BDE8BD0000F0B585B06A463C4BC6
:1032B0003C4913800F2301AF93700C310922380071
:1032C00007F01AF8FFF7F6FA374B384DC0182B689D
:1032D000984201D200232B602C68002C44D13E5D23
:1032E00001213000FFF7F4FA01340121300003F02E
:1032F0001FFA092CF3D100246B461E5D012130001A
:10330000FFF7E6FA01340021300003F011FA032C34
:10331000F2D1C82080000138C046C046C046C04631
:10332000C046C046C046C046C046C046C046C0466D
:10333000F1D100210520FFF7CBFA6B460021187868
:10334000FFF7C6FA6B4600215878FFF7C1FA6B46C3
:1033500000219878FFF7BCFAFFF7ACFA002413308D
:103360002860200005B0F0BDFFF7A4FA2B68002408
:103370009842F6D3052003F06BF80D4B0D4EC018A4
:103380000BD430603068032104F08EFE00230A4A1B
:1033900030602B6013600124E3E73460F2E7C0463D
:1033A0000D0E0000E8BD000010270000CC0F00202B
:1033B000C8FEFFFFB40F0020D40F002010B5012479
:1033C000044002D04410200010BD0D20FDF7BCFDCC
:1033D000F9E700000868F8B5C3071AD5FFF7EEFF54
:1033E0000300203B5E2B23D80520012258430023F5
:1033F000104E451DA84217D005211024375C3C42D1
:1034000000D09B180139520064100029F7D1013017
:10341000F0E704280CD90F2203681A40042A07D1C8
:103420001B0905D00079DBE701205B001843F8BDDC
:103430000120FCE7FDBD00000022054B10B51A601D
:10344000044B1B68934201D002F0AAFA002010BD81
:10345000D00F0020981A002070B508680D00FFF703
:10346000ADFF04006868FFF7A9FF621E0100042A8F
:1034700014D8451E042D11D805236B439B18012237
:1034800015009D402B00064805682B430360054B43
:103490001B68002B02D0200002F083FA002070BDD0
:1034A000D00F0020981A002070B508680D00FFF7B3
:1034B00085FF04006868FFF781FF621E0100042A8F
:1034C00013D8451E042D10D805236B439B180122E9
:1034D0009A400748036893430360064B1B68002B20
:1034E00003D00022200002F05CFA002070BDC0462C
:1034F000D00F0020981A0020F0B5050089B00868A8
:103500000C00FFF75BFF0690022D36DD6068FFF7C9
:1035100055FF0190A068FFF751FF04000127231D0C
:10352000661E0793731C0293079B9E4235D00523AA
:1035300073430593019B019D05330493049BAB42A8
:103540001ED0042E16D86B1E042B13D80122059B07
:103550002349013B5B199A409446224A0B68106844
:10356000069A3A4003920DD062461A430A6001223D
:1035700000280DD17F000135E0E701240194CDE75B
:10358000029ECFE7624693430B600028F2D0039A75
:103590000299280002F005FAECE7019B1E1D042E9B
:1035A0001AD8012C18D1002505273B0021006B43B8
:1035B0009B1999400B000A4A013511689943094B40
:1035C00011601B68002B05D0019B0022581D2900AB
:1035D00002F0E7F9052DE8D1002009B0F0BDC046A2
:1035E000D00F0020981A002010B5041E10DA1A24FB
:1035F0000A4BA400E25801239340094A0949136089
:10360000094A1160094A0A4911600A4A136010BD4B
:10361000FFF75CF9A042EADDEAE7C04670CA0000A5
:10362000C80F002008050050C00F0020BC0F00206C
:103630000C050050180500502B4BF7B51B680C000B
:10364000002B03D101204042FFF7CEFF2468012662
:10365000250035401AD0FF2263101202601210407C
:10366000DAB21043FF221B021204134018431F4B0F
:103670001B68202B06D1B4401D4BA40EA400E358B8
:1036800000021843FFF7C2FD0020FEBD042CFBD949
:103690000F2322681340092BF6D1FF2763683F02EE
:1036A0005B100193019B9D42EEDAAB00E3189B682F
:1036B000334216D05A105812D1B238400843FF2175
:1036C000120209040A401043084A1268202A06D14F
:1036D0005B009B0E06499B00020258581043FFF7FF
:1036E00095FD0135DEE7C046C80F00200800002028
:1036F000D8BF00000200086810B5C3070FD54010FE
:103700001823012A03DD4A68042A00D10833054A38
:103710001360FFF7FDF8FFF767FF002010BD0120E1
:103720004042EDE708000020086810B5C30703D544
:10373000FFF744FE054B1860054B1B68002B03D0B8
:10374000024B186802F02EF9002010BDD00F0020A7
:10375000981A00207FB5A04C2368002B0AD19F4AFD
:103760001268002A06D19E4B1B68002B01D0FFF780
:103770009BFD7FBD9B4D2A68002A26D1984A12687E
:10378000002A1BD0FFF790FD0028F2D0FFF778FD4C
:10379000924B24681A681C60002A16D0002C14D1A1
:1037A00001AD0C229049280006F0A6FD285D0021FD
:1037B0000134FFF78DF80C2CF8D1DAE7874A12684C
:1037C000002AE5D1002BE3D0E0E700210D2002F034
:1037D000AFFF00210E2002F0ABFF00210F2002F00E
:1037E000A7FF2E68012E5DD0022E00D1A2E0002E90
:1037F00051D101363100794C04202368994302F0FD
:1038000097FF04212368052019404B42594102F0DB
:103810008FFF10212368062019404B42594102F0C6
:1038200087FF80212368090119404B4259410C2030
:1038300002F07EFF80212368090219404B42594162
:103840000B2002F075FF80212368490219404B428A
:1038500059410A2002F06CFF802123688902194037
:103860004B425941092002F063FF80212368C902BD
:1038700019404B425941082002F05AFF8023216829
:103880001B0319404B425941072002F051FF310000
:103890000D2002F04DFF2B680321581C04F0EAFCB8
:1038A000296066E702214D4C0720236819404B42EE
:1038B000594102F03DFF0820216801404B42594127
:1038C00002F036FF80212368C90019404B4259415C
:1038D000052002F02DFF80212368490119404B4249
:1038E0005941062002F024FF80212368C9011940B4
:1038F0004B425941042002F01BFF802123688903B9
:1039000019404B4259410A2002F012FF80232168DE
:103910001B0419404B425941092002F009FF3100B4
:103920000C2002F005FF31000B2002F001FF3100F6
:103930000E20AEE72021294C0720236819404B4276
:10394000594102F0F5FE40212368082019404B42FE
:10395000594102F0EDFE80212368092019404B42B5
:10396000594102F0E5FE80212368490019404B428D
:1039700059410A2002F0DCFE8021236889001940A9
:103980004B4259410B2002F0D3FE8021236889016C
:1039900019404B4259410C2002F0CAFE8021236895
:1039A000490319404B425941062002F0C1FE8021D3
:1039B0002368C90319404B425941042002F0B8FE64
:1039C000802321685B0419404B425941052002F0D5
:1039D000AFFE01210F205CE7D00F0020C40F0020B4
:1039E000D40F0020B80F0020E8BD0000012010B562
:1039F0004042FFF7F9FD0020FFF708FC10BD000072
:103A000010B5034A0921034800F074FF10BDC046F9
:103A1000D8C0000020C1000030B502248025094B29
:103A2000094AED009C505C59002CFCD0A124E40014
:103A3000884202D30021995030BD8025ED001851F5
:103A40004019F5E700E001400405000010B500282A
:103A500006D1C020B02140028902FFF7DDFF10BD72
:103A6000B02080218002C902F7E70000434258419C
:103A7000064B40421840B0239B02C0180368002048
:103A80001A0E532A01D11B02180A704700C0FEFF0C
:103A900030B501248025054B054AED009C505C594A
:103AA000002CFCD001600021995030BD00E00140A5
:103AB0000405000043425841074B40421840B023E0
:103AC0009B02C018A62310B50902DB05090A194399
:103AD000FFF7DEFF10BDC04600C0FEFF70B5012439
:103AE00080250D4B0D4EED009C515C59002CFCD0F7
:103AF000002902DC00229A5170BD557814782D02FD
:103B000025439478013924042543D47804322406CB
:103B10002C4310C0ECE7C04600E001400405000063
:103B200070B505004B680A009C1C2100A400FFF73B
:103B3000D5FF281970BD0000134B1B68002B0CD05B
:103B40008022B023D2029B0200280BD11A1D5B6891
:103B50001B0E522B00D110007047B022C0239202DE
:103B60005B02F1E782420DD903681B0E522B09D18B
:103B7000436802339B00C018824203D903681B0EBE
:103B8000522BE9D00020E7E7D810002070B50020C4
:103B9000FFF7D2FFFF260500002801D1280070BDE5
:103BA00003681C143440FFF7C7FFDA2CF4D105007A
:103BB000F2E700008022F0B55200A1B00021674872
:103BC00006F0B6FB802200215200654806F0B0FBEB
:103BD000644BFF271B681A00049353425A4110009C
:103BE0000592FFF733FF049C0020631E9C415E4B4F
:103BF00064421C405D4BE418FFF7C8FF0600002E2E
:103C00002DD10498FFF732FF411C0598FFF752FFB2
:103C1000059A574D534B2C601A60FEF7CDFF514B60
:103C200064201B68A0215A4253414F4A5B42134013
:103C3000B0222C6892029B18E41A6043490204F0F7
:103C400033FAA0225202030000924A49220007A838
:103C500006F0B2FE07A801F067F821B0F0BD3268A7
:103C6000131412123A403B4003921A000A3A092AEE
:103C700049D83A4B039A995C002931D110223E4829
:103C800006F056FB35002B6803991A123A40914210
:103C900009D11A143A400B2A27D0132A2DD00A2A08
:103CA00001D1354B1D602800FFF746FF051EEAD104
:103CB000314B196800290FD02000FFF731FF0400B5
:103CC0002D4B5B195968002903D02000FFF728FF0E
:103CD000040004350C2DF3D1204B0121039A995493
:103CE0003000FFF729FF060089E73B40022BDADCB2
:103CF000214A9B00D3185D60D5E7102200211E48A1
:103D000006F016FBCFE71A00153A082AE8D8144A3D
:103D10000399525C002AE3D13500152B00D0150021
:103D2000300003681A143A40152A0FD01D2A00D11A
:103D30000025FFF701FF0028F3D1002D04D020005B
:103D40002900FFF7EDFE0400054BC6E7039A1B129E
:103D50003B409A42EDD10500EBE7C046D80F00206A
:103D6000E0100020D810002000C0FEFF04C00200B8
:103D7000DC100020B9C10000D42E0020F0B50020D6
:103D8000B7B00024FFF7D8FE270005002600002D5D
:103D90002ED1284D2868FFF769FE32003B000190C4
:103DA0000094254904A806F007FE04A800F0BCFF13
:103DB000224B64201C682B68A0215A425341204AA0
:103DC0005B421340B02292029B18E41A60434902FE
:103DD00004F06AF9A022520203000092194922005D
:103DE00004A806F0E9FD04A800F09EFF37B0F0BD7E
:103DF000FF226B6829689C460233FF180B120136BC
:103E000013409C4200DA1C00FF200A140240039277
:103E10006246014001920091039A0B4904A806F002
:103E2000CBFD04A800F080FF2800FFF785FE050009
:103E3000ADE7C046D81000202AC20000DC100020E8
:103E400000C0FEFFD4C1000016C2000070B5002003
:103E5000FFF70CFE04000120FFF708FE844200DAA1
:103E600004000A4B1D686A42554128001D60FFF797
:103E7000EDFDA0226B4252021340054A28009B1818
:103E8000044A611C1360FFF715FE70BDD8100020B6
:103E900004800100DC100020F8B50020FFF7E6FDEB
:103EA00007000120FFF7E2FD3E00204D0643204CB5
:103EB0000DD18021C020C9024002FFF7ADFD0121D4
:103EC0003000FFF7F7FD1B4B2E6023601DE087429B
:103ED00009DD0023B0212B60164B89022360236883
:103EE0000020012517E0012380212B60124BC9021D
:103EF0002360F4E7120E522A08D0002800D0236075
:103F00000E4800F011FFFFF7A1FFF8BD28005A6826
:103F1000023292009B188B4205D21A68561CE9D1D6
:103F20000028F2D0D1E72160EFE7C046D81000208A
:103F3000DC1000200480010004C00200EFC100007A
:103F4000F0B585B0039203220333DC17294D1440EA
:103F5000E4182B68284F5A42534180225B42D20218
:103F6000A4103B409B18A21C0291244E910000918A
:103F70000190316800980A18934215D2FFF71AFE93
:103F80002B685A42534180225B421F40D202BF1825
:103F90003368009A9B189F4206D2194800F0C4FE6D
:103FA0000025280005B0F0BD029B356819066B4658
:103FB0001A7BA423DB051343FF222F00090C1943AE
:103FC000019B12041B04134019432800FFF760FDF6
:103FD0000837281D21003760FFF75AFD002C04D058
:103FE0000A9A21003800FFF779FD009B083BFF1873
:103FF0003760D6E7D810002000C0FEFFDC1000209C
:1040000093C1000010B5FFF7D5FD10BD70B59AB093
:10401000FFF742FFFF221E4CD2000021200006F0D5
:1040200087F9FF25FFF7B2FD0026002814D1020012
:10403000C300E3580130591E8B41D218FF28F7D135
:10404000144901A806F0B8FC01A800F06DFE124862
:1040500000F06AFE1AB070BD03681A142A400A2ADA
:104060000AD11A122A40FF2A03D0D200A1180B71DC
:10407000A050FFF761FDD8E7132AFAD11B122B409D
:10408000FF2BF6D0DB00E2181671E650F1E7C046D0
:104090004C2500205FC2000073C200000021094BC4
:1040A000094A59600131516059680029FCD000214A
:1040B0001961012393600222044B8131FF315A5070
:1040C0001A607047FC1000400010004000E100E062
:1040D0000222064B0121DA670022054B5A61054A8C
:1040E00011615A69002AFCD07047C04604E100E023
:1040F000FC1000400010004010B5044C2378002B49
:1041000001D0FFF7E5FF0020207010BDE111002075
:104110000120024B1B685B001843704764120020AB
:1041200003480368002B02D1142203710260704718
:10413000FC2E00200120024B1B685B0018437047D7
:104140000C00002070B504000D001600FEF7B2FB55
:104150008023012200215B055B6E6270E270020A1F
:10416000A271020CE2711A0A60716372000EA272EF
:104170001A0C1B0E26702571A1702072E272237337
:1041800070BD0000124B10B51B68124C5A1C0FD0AA
:10419000114C002B0CD0114C012B09D0104C022BD0
:1041A00006D00D4C042B03D00E4C052B00D10B4C2C
:1041B00021000D4806F038FC200006F03DFC03000D
:1041C000042204339B0809481B011343036010BDFC
:1041D00010000020FBC20000F4C2000006C3000073
:1041E0000BC3000000C30000E82E0020E42E0020D6
:1041F00070B5214C2278002A3DD1204B01215A6014
:104200008022D20511605A68002AFCD000220720C3
:104210001B4B1C4901255A500439585008315A503B
:1042200019481A4958501A491A485A501A495A50A6
:10423000A622D2009D50082218495A5004315850E5
:104240000220174958501749174858501748043941
:104250005850182016495850C12189005A50053924
:10426000FF395858921802435A501249124A99502D
:10427000FFF714FF257070BDE1110020FC00004025
:10428000001000400C050000746962751C050000F8
:1042900024050000200004022C0500001405000085
:1042A000340500003C050000FFFF00002110010064
:1042B00054050000E21100200405000070B50E4B0B
:1042C00006001B78002B01D1FFF792FF00200B4D59
:1042D0002C7884420ED00A4B202219780323091B24
:1042E0001940084B4901C918300006F005F80120B3
:1042F000013C2C7070BDC046E11100206812002006
:10430000E0110020E2110020002370B588B098422F
:1043100027DD0D6801262C0034409C4221D123006A
:10432000042D1ED90F222B681A402300092A18D108
:104330006A681F2A15D96846FFF7C0FF23000028C6
:104340000FD06B4619783300A14203DB6B461B5D2F
:104350005B003343A200AA1801349360202CF2D1F1
:104360000423180008B070BD70B5414B8AB01B78AB
:10437000002B01D1FFF73CFF02AD2800FFF79EFFA5
:10438000002802D100200AB070BD2B780B2BF9D980
:104390006B78012BF6D1EB78012BF3D10023354E4E
:1043A000354C336023712B79344A1360002B0ED1C6
:1043B000152169444A780B7812021A438B781B0442
:1043C0001A43CB781B0613433360002318E0012BFC
:1043D00020D1152169444A780B7812021A438B7850
:1043E0001B041A43CB781A211B06134333600E2398
:1043F0006A7C6944934200DD130000229A4232D164
:1044000004200021E21804339B101B0103431171A7
:104410002360B8E7022B03D16A7B10331621E8E74B
:10442000042B0DD1152108226944684605F064FF6C
:104430000098019902F0EEF905F010FE3060C4E733
:10444000052BC2D1152108226944684605F054FFA6
:104450000098019902F0DEF905F000FE30606A7DF7
:104460000A231E21C5E78D5CA01805710132C5E73E
:10447000E111002064120020FC2E0020100000201A
:1044800010B5134B04001B78002B01D1FFF7B0FED1
:10449000FFF71EFE00200F4A0F49104B5450586082
:1044A0000130106058680028FCD0002018610130ED
:1044B000906018690028FCD0094B0A481B785B0102
:1044C0001B185350FFF704FEFFF7E8FD10BDC04670
:1044D000E11100200010004004050000FC10004025
:1044E000E0110020E211002010B588B000281DDD89
:1044F0000A68012113000B4018D1042A16D90F2095
:1045000014682040092811D150681F280ED998003E
:10451000101880680024084201D04010C4B26846D8
:10452000C4540133202BF2D1FFF7AAFF002008B0BA
:1045300010BD000010B5002813DD0C68E30710D58E
:104540006410532C0DD8084B1B78002B01D1FFF7BA
:104550004FFEFFF7BDFDA123044ADB00D450FFF757
:104560009DFD002010BDC046E1110020001000405C
:1045700010B500280EDD0C68E3070BD56410FF2C86
:1045800008D8054B1B78002B01D1FFF731FE034AF9
:10459000034BD450002010BDE1110020001000405A
:1045A0002405000013B5002814DD0C68E30711D5BD
:1045B000094B64100093094B0193072C0AD8084B50
:1045C0001B78002B01D1FFF713FE6B46054A1957E4
:1045D000054BD150002016BDE2ECF0F4F8FC0004CD
:1045E000E1110020001000400C05000070B588B0FB
:1045F000002820DD0124086804401CD104281AD9B1
:104600000F2302681340042B15D1FEF747FB060069
:1046100006F012FA0500122800D912252A000221FC
:104620000D326846FFF78EFD6B465D73A54205DCD3
:104630006846FFF725FF002008B070BD2300325DFB
:104640006B449A730134F1E7F0B50D008BB001288B
:1046500032DD08680122040014402DD104282BD932
:104660000F2301680B40042B26D16B68134223D023
:10467000FEF714FB6E6807007310019306F0DCF977
:1046800005000E2800D90E252A000121113202A8AA
:10469000FFF758FD6A46127902AB5A7302AA7312E9
:1046A0009373019B76141B0ED67313745574A54235
:1046B00005DC02A8FFF7E4FE00200BB0F0BD3A5D78
:1046C00002A963189A740134F1E730B589B0002863
:1046D00014DD0C68E30711D5102268460021FFF7AE
:1046E00031FD6B466A4665105D73684663122D0E98
:1046F00064149373D4731574FFF7C2FE002009B0DD
:1047000030BD0000174B184A5968002903D000211A
:10471000596001319160196900291FD0002018618A
:104720008023DB00D3581149012B18D1A923DB00CA
:10473000D3585B420B600E490B78032B01D8013331
:104740000B7003200B490B78013303400B700A49AF
:104750005B015B180949535001239360704708605F
:10476000FAE7C046FC100040001000400C0000209A
:1047700068120020E0110020E21100200405000072
:1047800010B5034A0E21034800F0B4F810BDC0462E
:1047900084C200007BC20000044A05491368C85463
:1047A00001339B059B0D13607047C04684160020A3
:1047B0008412002070B5114C114A2368834202DC38
:1047C0000023236016E0155C411C2E00FA3E012EEA
:1047D00005D899420FDA555C013D1F2D01D908001B
:1047E000ECE70100151A565C6E5401318B42FADC7D
:1047F000181A206070BD1570FAE7C046901A0020A4
:104800009016002010B5FEF74BF8064B1A6882424E
:1048100001D900221A601B68C31A034898428041DC
:10482000404210BD80120020204E000010B5094CFF
:10483000094A23681268934200D110BD074AD05C30
:10484000FEF7B2F90028F8D0236801339B059B0DD1
:104850002360ECE7881600208416002084120020D4
:1048600010B50400064B074A1B6812689B1ADB430D
:104870009B059B0DA34200DB10BDFFF7D7FFF1E7BF
:104880008416002088160020F7B5050056680191AF
:10489000B000441C06301700FFF7E2FFFB20FFF7D3
:1048A0007BFF1C20FFF778FFE8B2FFF775FFE0B24F
:1048B0002412FFF771FFE0B2FFF76EFF6B46187925
:1048C000FFF76AFF0025AE4200DCF7BDAB00FB1826
:1048D0009C680135E0B2FFF75FFF2012C0B2FFF71E
:1048E0005BFF2014C0B2FFF757FF200EFFF754FF05
:1048F000E9E7000070B5074E3368092B08DC0C258A
:104900005D43054C0133285164196160A260336036
:1049100070BDC0468C160020202F0020F0B587B057
:1049200002900C00012803DC1B20FCF70DFB45E086
:10493000244B08680093C30709D4042807D90F2320
:1049400002681340042B02D1FEF7A8F900901D4B1A
:1049500060680193C30709D4042807D90F230268AC
:104960001340042B02D1FEF799F901900027164B52
:104970001B680493049BBB42D6DD0C267E43134B7D
:104980000099F618306806F045F8051E05D17368E1
:10499000B6680593059B9D4201DB0137EAE7306865
:1049A0000199039606F036F80836002808D1210050
:1049B0000298039B083102385B68984707B0F0BD46
:1049C0000135E7E7EEBC00008C160020202F002008
:1049D00010B5FCF705FAFFF713F8FEF787F8FEF7B6
:1049E000C5FBFEF7FBFBFFF7CBFE00F027FE00F058
:1049F000DBFF10BD962210B512010021034805F01F
:104A000097FC0022024B1A6010BDC046EC1B002030
:104A1000B0050020064B074A1B6812689B1ADB434F
:104A20009B059B0D0122834200DC00221000704791
:104A30008416002088160020F8B505000C0016002A
:104A40001F1E0ED10320FFF7E5FF002808D0FA2033
:104A5000FFF7A2FEE8B2FFF79FFEE0B2FFF79CFE71
:104A6000F8BD501DFFF7D6FF0028F9D0FB20FFF757
:104A700093FEE8B2FFF790FEE0B2FFF78DFEF0B2D2
:104A8000FFF78AFE3012C0B2FFF786FE3C00E31B40
:104A90009E42E5DD2078FFF77FFE0134F7E7000056
:104AA00070B50024F0250B4B1B68A34202DCFFF716
:104AB000A1FF70BD2B006343074A9B181A78002A98
:104AC00005D05978002311201A00FFF7B5FF0134F3
:104AD000E9E7C046B0050020EC1B0020F8B5070050
:104AE0000024F0252B0063430C4A01349E18B74282
:104AF00011D0317800290BD00133D15C0023112073
:104B00001A00FFF799FF2A000021300005F010FC81
:104B10000A2CE7D1F8BD024B1C60F9E7EC1B002022
:104B2000B0050020FFB501231700FFB001900291EE
:104B300015001F4011D004AA13706B1004A9537004
:104B40006A128A7005221B0E6D140B71CD700B005A
:104B50000299FFF771FF7FB0FFBD042A1FD90F2311
:104B600012681340042B26D1023B04AA28001370BC
:104B7000FEF794F8040005F05FFFF823FF33984236
:104B800000D91800B84204DC421C04AB0299019819
:104B9000DFE701377B1EE35C04AAD355F2E7042A62
:104BA0007ED1032304AA043D13706B425D411300C0
:104BB00055700222EAE7092BCDD16946053B04AACC
:104BC00013706B685A1000925B1204AA09789370F4
:104BD000009B5170132B01DD142300936A46127859
:104BE00004ABDA7005AC009BBB4202DC04ABE21AFA
:104BF000CCE70126BB00EB189868064006D10428D4
:104C000037D90F2302681340022B0CD101232370E4
:104C10004310637042121B0E4014A270E0702371A7
:104C200005340137DFE7042B21D1023B2370FEF767
:104C300035F8039005F000FFA31C0C2809D860701C
:104C4000864201D19C19ECE7039A925D9A55013690
:104C5000F6E70C226270039A925D9A550136092E8E
:104C6000F9D12E23E372237363730E34D9E7012B3A
:104C700007D1032304382370434258416070023443
:104C8000CFE7092B09D1053B23704368E6705A1022
:104C90005B126270A3700434C3E726700134C0E76E
:104CA000002A00D057E77CE770B502000024F0210D
:104CB0000D4E0800604380194578954203D00134B9
:104CC0000A2CF6D170BDF022002105F031FB074A15
:104CD0001368013BA34200D11460002329001A008D
:104CE0001120FFF7A9FEEDE7EC1B0020B005002026
:104CF00010B5B2B002236A460400137005F09CFEA2
:104D0000C72800D9C7200023984207DC421C6B4605
:104D1000FE211420FFF790FE32B010BD694601332A
:104D20005A1EA25CCA54EFE730B5B3B002236A46FC
:104D30000500137005F080FE0400C72800D9C724C1
:104D400000239C420BDC20003230FFF789FD621CFF
:104D50006B46FF211420FFF76FFE33B030BD69466C
:104D600001335A1EAA5CCA54EBE70000F7B5234B87
:104D700006001B68F02100930023009A9A4211DC80
:104D80000024F0231A006243019201991C4A55182D
:104D90002F78002F12D001340A2CF3D11948FFF7D5
:104DA000C3FF29E00A005A43154882185078B042E0
:104DB00002D11278002A1FD10133DEE7F022390038
:104DC000280005F0B5FA02230D4A0199EB6053540F
:104DD0000D4AF1008A58009B6E70AE70AA602F6178
:104DE0006F61A34202DC054B01341C6000233100DB
:104DF0001A001020FFF720FEF7BDC046B0050020C6
:104E0000EC1B0020F5C700004C25002010B5FFF773
:104E100047FEFF24084AE3005B429B18074AD35C25
:104E2000043B012B03D8E043C0B2FFF79FFF013CD6
:104E3000002CEFD110BDC046FC0700004C2500201F
:104E4000F7B50E00FF247F2501901C4AE300D31A1A
:104E50001B4A9A181278062A01D0032A1DD1FF2274
:104E6000D2009B18186883682B401C2B15D1C3688F
:104E70001A002A40042A10D102692A40192A0CD1AA
:104E80001B0A01339B000C30C018FDF707FF070019
:104E900005F0D2FD0023B04209D0013C002CD4D152
:104EA000F7BD019AF95CD25C9142F6D101339E4282
:104EB000F7DCE043C0B2FFF759FFEEE74C250020D6
:104EC000FC07000070B50500FF24084AE3005B42C0
:104ED0009B18074AD35CAB4203D1E043C0B2FFF753
:104EE00045FF013C002CF0D170BDC046FC0700001E
:104EF0004C250020F7B5FDF7D3FC514B1A688242D0
:104F000001D900221A601A684E49821A8A4200D8D2
:104F100083E01860FDF7CEFC071E00D101370020AA
:104F2000FDF7BAFD01900020FDF7CAFD019B00903E
:104F3000454C464D002B14D02368002B00D07AE05E
:104F40002B682760002B00D171E0414B01261B78B4
:104F5000002B63D10920FFF7B5FF3E4B1E703C4B81
:104F60001E70009B002B12D02B68002B0FD12368E2
:104F70002F60002B1ED0374B01261B78002B52D1FF
:104F80000920FFF79FFF334B1E70314B1E702368C3
:104F9000002B0FD02F4E3278002A0BD19F4200D227
:104FA00027602368FB1A312B04D90720FFF78AFFFB
:104FB000012333702B68002B0FD0254E3278002A46
:104FC0000BD1BB4200D92F602B68FF1A312F04D9B7
:104FD0000820FFF777FF012333702368002B0CD0E4
:104FE000019B002B09D11B4E3378002B02D10720E7
:104FF000FFF768FF0023236033702B68002B0CD071
:10500000009B002B09D1124C2378002B02D10820E1
:10501000FFF758FF00232B602370F7BD0720FFF731
:1050200051FF0C4B9CE70820FFF74CFFADE7009BBE
:10503000002B9CD1ABE7009A002A95D1AAE7C04685
:105040007C1200200F2700006C1200207412002038
:10505000781200207012002037B500240500FFF7F9
:105060001FFD01A80194FDF705FD21002000FEF7BA
:10507000E3F9FEF76FFBFDF737FDFDF736FDFEF7B1
:10508000B5FCFDF733FCA54204D0FDF7B7FD02489F
:10509000FFF74AFE37BDC046E6C70000002310B543
:1050A00001001A001120FFF7C7FC10BD07B56B46C1
:1050B000197069465A7013128B701314120ECB704C
:1050C0000A716B46010005221320FFF7B5FC07BDEE
:1050D00010B50A0001001220FFF724FD10BD70B5C5
:1050E000050008000C003230FFF7BAFB2B0022004D
:1050F00000211B20FFF7A0FC70BD10B50C000300C1
:10510000110014202200FFF797FC10BD012370B599
:10511000FF24084A41185B42884201D3D84370BD3E
:1051200006781D0A234073409B009B5801306B405A
:10513000F2E7C046C8C30000002313B501930B4B30
:10514000C2000400D058002805D0436808309900F8
:10515000FFF7DCFF01900920FFF782FB01AB04227F
:1051600021001720FFF768FC13BDC0464C25002026
:1051700070B506000020FEF7DFFC0024FF250028A4
:1051800001D1200070BD03681A142A40152A07D1E6
:105190001B122B40B34200D10400FEF7CDFCEEE71A
:1051A0001D2AFAD10024F8E7F0B580279DB0FFF75B
:1051B0003DFBAD4CAD4D2068FF00391A4019FDF79D
:1051C000D9FC23680600C3182360002B0ED11DB044
:1051D000F0BD2068391A2818FDF7CCFC23680600BA
:1051E0001B182360FDF75CFBA14B1860002EF0DC60
:1051F0002B78FA2B00D013E12368022B07DCFFF792
:1052000001FB0028E3D00120FFF7D4FADFE768783C
:10521000AC78023818281FD802F0B2FE0D202428DE
:105220002B341E3E6872768CDEEF1E1E1E1E1E1E66
:105230001E1E1E1EFD00FF2C0ED02000FFF734FDA9
:1052400000228C4BE100CA505B181A7121000092B9
:1052500013001320FEF774FE0320D5E72000FFF7AC
:1052600085FDF9E72000FFF71FFDF5E7FFF7CEFD0D
:10527000F2E7FFF715FC0020FFF7EEFE7E48FFF790
:1052800053FDE9E7632CE7D87C4BA200D2582100FC
:105290001520FFF747FCDFE700242000FFF768FF39
:1052A000061E03D10134642CF7D1D5E7083005F090
:1052B000C3FB05000530FFF7D3FAFB20FFF76CFABC
:1052C0001D20FFF769FAE0B2FFF766FAE8B2FFF7D0
:1052D00063FA2812C0B2FFF75FFA3700BB1B9D428A
:1052E000E0DD387AFFF758FA0137F7E700211D2093
:1052F00000910B000A00FEF723FEFDF77FFCABE7F1
:105300002000FFF719FFA7E7FDF7DCFA03AC5C4AC2
:10531000642100905B4B200005F01CFB0223200061
:10532000237005F089FB2300020000211620FFF7FF
:1053300083FB91E700244F4AE300D558002D28D085
:105340006B689E00701DFFF78BFA2B000025320062
:10535000083321000120FFF76FFB0020FEF7ECFB74
:105360002F002E00002818D1002F04D03A00012170
:105370002000FFF789FA002D04D02A000221200026
:10538000FFF782FA002E04D0320000212000FFF740
:105390007BFA0134FF2CCED15EE7FF2103681A129D
:1053A0000A40A24209D11A140A400B2A08D10B4024
:1053B0000CD0012B0CD0022B0CD0FEF7BDFBD1E79B
:1053C000132AFAD100252F002E00F6E70600F4E795
:1053D0000700F2E70500F0E70024FFF761FB220079
:1053E000210000942300DA20FEF7AAFDFF2221000D
:1053F000D200204804F09CFF7FE7012C02D1FEF789
:10540000BDFC29E7022C02D1FEF7FCFD24E70120B8
:10541000FFF722FE20E7002321001A001A2086E76A
:10542000FB2B00D0EFE62268042A00DCE7E62E79A9
:10543000E878154B360206439E4200DDE3E6331D55
:105440009A4200DCDBE6EB5CFE2B00D0DBE66B78FF
:10545000AC78711E1B2B6BD018D8012B2BD0082BCE
:105460003DD0701DD0E6C046901A00209016002056
:10547000801200204C250020C8C70000442D0020C9
:10548000DFC70000DAC70000F60300001D2B60D064
:1054900052D31E2BE5D1012CE3D10029E1DD6B793C
:1054A000002B03D01C00322B00DD322464235C432C
:1054B000344B1C60D5E7FF2CD3D02000FFF7F4FB62
:1054C0006D79314AB31E009221002A000A20FEF7AE
:1054D00037FD2E4BE400E0501B191D71C1E7632C12
:1054E000BFD86A79022A13D0032A1BD0012AB8D167
:1054F000E979AB79090219432B7AA4001B041943FB
:105500006B7A1B060B435B001343214AA350A8E7A9
:105510000029A6DDB11E1C48FDF7C2FD1C4BA400EE
:10552000E0509EE7AB79A4005A1E93419B00ECE744
:105530001848FFF785FC94E7FF2C92D06A79022A7D
:105540008FD811490B2000912100B31EFEF7F8FC03
:1055500087E70B00632900DD6323002203A8934241
:105560000ADCD9430022C917194041180A700133D7
:10557000009021001520E9E7A918497981540132EA
:10558000EDE7C04604000020961600204C250020C0
:10559000442D0020951600200120704710B5064CC0
:1055A000200000F037FB0549200000F05BFB0122E2
:1055B000034B1A6010BDC046BC1A0020801A0600BA
:1055C000941A002010B501210D20FDF781F9012169
:1055D0000E20FDF77DF900210F20FDF779F9044C2D
:1055E000200000F053FA1021200000F06BFA10BDEB
:1055F0009C1A002010B504680D20E30703D5641041
:10560000FF2C03D91720FBF79FFC10BDFFF7DAFF33
:10561000E1B2024800F078FA0020F6E79C1A002078
:1056200010B5FFF7CFFF0021034800F06DFA4300EB
:105630000120184310BDC0469C1A002010B5034A33
:1056400008210348FFF756F910BDC0460CC80000FA
:105650004CC80000F8B5012306681E4205D0456815
:105660001D4202D084681C4203D10D20FBF76CFC64
:10567000F8BD76101520802EF8D86D101620FF2D5D
:10568000F4D86410FF2C01D91720EFE70B4B1B68EF
:10569000002B01D1FFF782FF094FF1B2380000F073
:1056A00078FBE9B2380000F07BFAE1B2380000F094
:1056B00077FA380000F0D8FB0020D9E7941A0020D0
:1056C000BC1A0020F7B501242300A0421DDD0D689F
:1056D0002C421AD01A4B25411B684C68002B01D173
:1056E000FFF75CFFE9B201272500164E3D40300070
:1056F00000F04FFB002D0AD03C413000E1B200F039
:105700004FFA300000F0B0FB00231800FEBD042C5F
:10571000F7D90F2322681340092BF2D163685B107D
:105720000193019BAB42ECDDAB00E3189968394271
:1057300004D04910C9B2300000F032FA0135F0E768
:10574000941A0020BC1A0020144B70B51B68050089
:105750000E00002B01D1FFF721FF114CEDB2290003
:10576000200000F016FBF1B2200000F019FA002131
:10577000200000F019FB002801D0404270BD01223A
:105780002900200000F000FB200000F0FAF90028BA
:10579000FAD0200000F0FAF9F0E7C046941A002091
:1057A000BC1A002010B501240368234202D04168CE
:1057B000214203D10D20FBF7C7FB10BD58108028F4
:1057C00001D91520F7E74910FF2901D91620F2E782
:1057D000FFF7BAFF40002043EFE710B504000128AF
:1057E00014D105211820FFF7AFFF7F282BDC030021
:1057F0007F3301DA7F20404264235B4258437F219C
:1058000002F052FC052C00D1404210BD032811D1FA
:1058100001001820FFF798FF7F2814DC03007F3376
:1058200001DA7F20404264235B4258437F2102F02B
:105830003BFCEAE70020052CF5D107211830FFF7E3
:1058400083FF7F2802DD0138FF38D0E703007F3374
:1058500001DA7F20404264235B4258437F2102F0FB
:1058600023FCD1E770B50120FFF7B7FF0400032048
:10587000FFF7B3FF05000520FFF7AFFF6D4364435B
:1058800040436419201804F01FFC01F0F3F804F001
:10589000E5FB43000120184370BD10B50120FFF760
:1058A0009CFF43000120184310BD10B50320FFF7F3
:1058B00094FF43000120184310BD10B50520FFF7E9
:1058C0008CFF43000120184310BD10B5082118209B
:1058D000FFF73AFF0300C00FC01801234010153036
:1058E0004000184310BD0000F8B501231C00984289
:1058F00034DD0F683B4231D04E6835001D402DD15C
:10590000042E2BD90F2231680A40092A26D1736848
:105910005C10202C00DD2024114B1B68002B01D1D2
:10592000FFF73CFE7F10F9B20E4F2200380000F066
:105930002BFAA5420FDA380000F023F90028FAD03C
:10594000380000F023F90122AB004000F3181043A7
:105950009860AD18EDE70120640004432000F8BD15
:10596000941A0020BC1A00200020704701207047C4
:1059700000207047002070470120704700207047CA
:1059800000207047002070470020704700207047BB
:1059900000207047002070470020704700207047AB
:1059A000704770477047000010B5034A0E21034846
:1059B000FEF7A0FF10BDC0469CC800000CC9000047
:1059C00010B5FDF79FF8FDF73BF9FFF701F8044824
:1059D000FFF7AAF9FEF71AFBFFF718FA10BDC04649
:1059E00095C9000010B5FCF7F5FE10BD70B5002597
:1059F00004AC24780573A94205D10A4B0A4A232135
:105A00000A4804F00BFC01600949920052589B00BF
:105A100002715B58A400837163588560437102234F
:105A2000C37170BDADC9000012CA0000BBC900003F
:105A300070CA0000037B002B04D14373837303619E
:105A400001330373704700001FB50191A0210024AA
:105A50000068C900D2B24450012A10D0A24209D035
:105A6000032A0AD0074A8350074B019AC2500123E8
:105A700043501FBD02221343F4E70422FBE7062232
:105A8000F9E7C046540500002405000010B50400E5
:105A9000FFF7D0FFA1222368A179D2009950617944
:105AA000064A20009950217904329950044B196814
:105AB0005A689B68FFF7C8FF10BDC0460C05000080
:105AC000B01A00204BB2002B0FDB80233F290FD8E8
:105AD0001F290FD80F290FD807290FD803290FD84E
:105AE0001B060168074A8B50704780239B04F8E728
:105AF000DB04F6E71B05F4E75B05F2E79B05F0E73F
:105B0000DB05EEE7240500000368074A99501A00F8
:105B1000FC32D1680029FCD0A321C90058580023C9
:105B2000C0B2D3607047C0461C05000007B5802294
:105B3000074BD2051A6000229A6002321A711123B3
:105B40000E320093034905330348FFF74FFF07BDAB
:105B5000B01A0020003000409C1A0020F8B5050063
:105B60000E0017000024BC4208D02B68315D1B6872
:105B700028009847002801D00134F4E72000F8BD40
:105B8000704710B51C3000F0A9F910BD10B51C30DD
:105B900000F096F910BD10B51C3000F0A5F910BD4D
:105BA00070B5437E0D00002B01D1002070BD643024
:105BB000040000F0A2F90028F7D12000290000F02D
:105BC00070F90120F2E70000F7B50193FA230025F0
:105BD00004009B0083600D4B4560083303601C305C
:105BE0000F00160000F052F92000643000F04EF96A
:105BF000074A2761B600B35820006375019B9B00DC
:105C00009B586576A576A375FEBDC04650CA0000B8
:105C100070CA00000123A022C375837D0E49C133E1
:105C2000FF33D2059B009950437DC133FF339B0066
:105C30009950CC220169094B5204CA5005220169CE
:105C4000243BCA50827D01690833CA500269417DF4
:105C5000034BD1507047C0460C06000024050000DD
:105C60000C050000A022002310B50469D200A35047
:105C70000A4CA1420FD90A4C8C425B4109495B4254
:105C80000B40CD21C9045B18046907496350052105
:105C90000369995010BDCC235B04F5E7A086010091
:105CA00090D00300000098FD24050000F7B5040023
:105CB00000200D000193824265D01600402A00D9D1
:105CC000402627001C37380000F0F6F8B12322697F
:105CD000DB00D55080220123216992008B50A27EE7
:105CE000002A03D122691362226913600025731E02
:105CF000AB4207D1019B002B04D0802202212369F3
:105D000092009950012223691A622369FC33DA68F0
:105D1000002A02D19A6A002AF9D09A6A002A0BD185
:105D2000DA60A3232269DB00D1583800C9B20135FB
:105D300000F0B7F8B542DAD3019B2269002B0FD1EE
:105D40001300FC339B6A002B0AD10133A376D36185
:105D50002369FC33DA6C002AFCD00022DA640AE002
:105D600000230121A37651611A002369FC3399684D
:105D70000029FCD09A602369FC339A6A002A01D07A
:105D800000229A62E8B2FEBD10B50123FFF78EFF34
:105D900010BD0300AC3310B504001970643000F07E
:105DA0008BF80123637610BD0023020070B5AC327E
:105DB00043760D001178B12204000069D2008150B1
:105DC0008022216992008B5022690133136222697B
:105DD000936026006436300000F080F8002812D06E
:105DE000300000F06DF81E4B2269D0502369FC335F
:105DF0001A6A002A02D19A6A002AF9D09A6A002AFD
:105E000001D11A62E5E723690122002D0DD11900A5
:105E1000FC31896A002908D1DA612369FC33DA6C24
:105E2000002AFCD00022DA6407E05A612369FC33BF
:105E30009A68002AFCD000229A6000202369FC3373
:105E40009A6A82420BD098622169064A8B588B501D
:105E50001800022B03D0181F431E9841033070BD59
:105E60001C050000C404000010B50121FFF79CFFD1
:105E700010BD000010B51323122202490248FFF79B
:105E8000A3FE10BD00400040BC1A002010B5402207
:105E90000021040004F04CFA002320002364636412
:105EA00010BD10B53F24026C531C2340446C9C422F
:105EB00001D08154036410BD002303644364704720
:105EC000436C026C934206D03F21C25C01330B400D
:105ED00043641000704701204042FBE7036C406CB4
:105EE000181A00D540307047436C026C934201D0C1
:105EF000C05C704701204042FBE73F22036C406CCE
:105F000001331340181A43425841C0B27047000091
:105F100003210A4802680A430260094802680A43EA
:105F200002600849084A094B9B1A03DD043BC85824
:105F3000D050FBDC00F012F8FAF7E6F82405004038
:105F400054050040BCCF00000000002048020020A3
:105F5000FEE7FEE7FEE7FEE7FEE7FEE72D4B10B5A6
:105F60001A68D2B2012A0FD12B4A126812070BD13C
:105F70002A4AE0241168F0220800104021422DD165
:105F80002749096811422CD01A68D2B2012A12D1CD
:105F90002149096809070ED1F0202049096801400C
:105FA000402908D11E490968014204D18020C1213D
:105FB000C005C90042501B68DBB2012B0DD1164B46
:105FC0001B681B0709D1154B1A68F0231A40A02A39
:105FD0000FD1134A12681A420ED010BD3028CFD00C
:105FE000D2E7104A104911608021104A090211605D
:105FF000CAE7D02AF1D1ECE70D4B1A68012A04D088
:106000000C4A1A601A68012AFCD1C0220A4B1A6095
:10601000E3E7C046E00F00F0E40F00F0E80F00F007
:10602000EC0F00F004050040DFFF07C0186C0040D3
:1060300000EC06407593000014EC06400120704708
:1060400010B503681322DB69984710BD7047000044
:10605000054B0269D1500369FC331A6A002AFCD04F
:10606000002201201A6270471C050000030010B5D1
:106070005C331A781F231A401E3B19009140114AC5
:10608000D167C222042104699200A15002695360C1
:106090000269D360A02300220169DB00CA500123FA
:1060A0000169094A5B428B500169084A8B500169BA
:1060B0000C3A8B50016908328B501430FFF7FCFE0C
:1060C00010BDC04604E100E00C050000140500000E
:1060D00010B51430FFF702FF10BD10B51430FFF7F4
:1060E00003FF10BD10B51430FFF7EAFE10BD00002D
:1060F000030070B55E331A780469724BE2500300F6
:106100005D331A780469704BE250030061331C78E8
:1061100002696E4B012C00D09EE005005F352E78A1
:10612000A225ED005651020060321578A1220669C1
:10613000D200B5500269D4509623DB00994200D8B2
:106140008CE096231B01994200D88AE096235B01DC
:10615000994200D888E096239B01994200D885E0B7
:10616000E1239B01994200D882E09623DB0199420A
:1061700000D880E0E123DB01994200D87DE096233E
:106180001B02994200D87AE0E1231B02994200D811
:1061900077E096235B02994200D874E0E1235B022A
:1061A000994200D871E0E1239B02994200D86EE049
:1061B000474B994200D86CE0E123DB02994200D8BA
:1061C0006AE0E122002312038A425B41414A5B42BA
:1061D0001340802252059B1801693F4A8B50A0232F
:1061E00004220169DB00CA5000210369FC33D96035
:1061F0000369FC331962012301690B6001698B603B
:10620000C1210469890062501F215C3002780A4074
:1062100093406231314AFF315350002141560029E9
:106220003CDA0F230B40083B2D4C9B089B001B19AD
:1062300003242140A140FC348C40DD69A5432C009F
:10624000C0258D4029002143D9611F2301781940C1
:106250001E3B8B40136070BD00246CE79E23DB0265
:10626000BAE79D231B03B7E71E4BB5E71E4BB3E709
:10627000EC239B03B0E71D4BAEE71D4BACE71D4B7A
:10628000AAE71D4BA8E71D4BA6E71D4BA4E71D4B36
:10629000A2E78023DB049FE71B4B9DE78C080F4B95
:1062A000A400E41803230B40FF21C025DB00994024
:1062B000AD0066598E433100C0269E4033000B432B
:1062C0006351C2E70C050000140500006C050000D6
:1062D00090D0030000D0BEFE2405000000E100E0E5
:1062E00000ED00E000B013000050270000A04E00B9
:1062F00000F0750000509D0000F0EB0000903A01A6
:1063000000E0D70100B0AF0300705F07F7B500935E
:1063100008AB1B7800250193FA2304009B008360DF
:106320000E4B45600833036014300F001600FFF772
:10633000ADFD23005C3327611E70009B084A9B0063
:10634000995823005D331970019B20009B009A58D7
:1063500023005E33DD701A70FEBDC046ECCA00003B
:1063600070CA0000036910B51A00FC32D26804003C
:10637000002A0AD0A322D20099581430C9B2FFF7DC
:1063800090FD00222369FC33DA6010BD10B502488D
:10639000FFF7E8FF10BDC046741B00201D2307B5A2
:1063A00002220093024901330248FFF7AFFF07BD05
:1063B00000200040741B002010B5002801D004F01C
:1063C00073FA10BD7047000010B500F011F8FFF728
:1063D000F9FF012000F000FAFFF7F2FAFFF702FBE5
:1063E000024B002BFAD000E000BFF7E700000000EE
:1063F000C420114B80001A5810491140C0221202CB
:106400000A431A50C0218022490092025A501A6051
:106410008023A3220021DB05D20099500122F9300C
:106420009A60074BFF301950C1200231800019508B
:10643000403019501A60704700E100E0FF00FFFF94
:1064400000100140014B18607047C0465C000020FE
:10645000F7B500231E285AD8384B8000C258042AAA
:106460005BD007D8022A54D055D80423012A09D07A
:1064700000234CE0062A54D051D31A2A53D00223C9
:106480001B2AF5D12E4A116808294ED909294FD067
:106490000A240226A02001252A4AC00015502A48B5
:1064A0002A4D07681C20BF00074029480197006853
:1064B0005759009027481B0207401F43C0230098EC
:1064C0009B020340FF2057515759000207401F43CA
:1064D000019B1F43009B58016023184007433E4324
:1064E000565101251C4B156058680028FCD000202F
:1064F0005860A1230125DB00D3585560A025ED008D
:1065000050511BB2A14202D015D2611ACB401800E3
:10651000FEBD0823B6E71023B4E72023B2E74023EB
:10652000B0E78023AEE70123ACE708240026B1E7FB
:106530000C000126AEE7091B8B40E8E770CA00009B
:1065400058000020007000401400002004050000E6
:1065500018000020FF00FFFFFC700040F0B51E286F
:106560005BD8364B8000C258354B1E68002E30D1A8
:10657000C227344BBF00D859334C03250440C020F8
:1065800000022043D851C0248020640080001851AC
:106590002E4F18602E4B803CD859FF3CA043D85159
:1065A0000437D859A8432043D8510837D8590C3557
:1065B000A8438446072065462843D851A820C00038
:1065C0001E50C1208026800076021E501C601C4B8D
:1065D0001C60142500202B001E4C2E00464336590B
:1065E000771C1BD14343E250A0230325C132FF3265
:1065F0009200DB05D550184B1A68082A14D11423D1
:106600004343E3189A6812485132FF3292005960AE
:106610001150DA68C1239B00C250F0BD9642E1D010
:1066200001300328D9D1F8E7082A02D9083AD14025
:10663000E5E708239A1A9140E1E7C04670CA0000D6
:10664000D81B002000E100E0FF00FFFF0405000070
:10665000009000401C0000205C0000202149F0B5A3
:106660004A6C2148002A14D0A025A1260023012429
:10667000ED05F600C258571C06D0C7187F68002FDA
:1066800002D027009740AF5114333C2BF2D10023A6
:106690004B64A0230121DB0500260F009C46142338
:1066A0004B43C3181A1F1268104C0E4D9200141958
:1066B0005219526C002A10D01A00143A1268551C54
:1066C00009D0103B1B68FF2B05D03B00934065466B
:1066D0001A00074BEA50FC34666401310429DED10C
:1066E000F0BDC046FC9000401C000020009000401F
:1066F0000C05000000B51E2810D80C4A80008358F5
:1067000003290BD8A0220800C133FF33D2059B0018
:1067100001F036FC020905070021D15000BD0C2113
:10672000FBE70421F9E70321F7E7C04670CA000040
:106730001E280AD8074B8000C25801239340A0228C
:10674000D205002902D1044953507047A121C90044
:10675000FAE7C04670CA00000C05000003000020E4
:106760001E2B0AD8A021A222C905D2008858034AAC
:106770009B009B58D84001231840704770CA000006
:10678000F7B506000D000C008B180193019B671BE9
:106790009C4207D0336821781B6830009847013449
:1067A0000028F3D13800FEBD0849094A094B10B54D
:1067B0001B688858FA22190A1B0618439200002306
:1067C00001F0AAFD4904C00B084310BD00100140B0
:1067D00004050000DC1B002070B5041E09D0FFF783
:1067E000E3FF050000F014F8FFF7DEFF401BA042B6
:1067F000F8D370BD0022044B9A60044A1368013339
:10680000DBB213607047C046FC100140DC1B002067
:1068100070470000F0B5C64600B5CB0F9846404A19
:106820004B005B0D9A1882B00D000400132A2FDC78
:10683000002A49DB3B4F17413E000E40064323D060
:106840007F08390029400C430AD03749BD438C46A4
:1068500063445C425C418023DB021341E4071D4337
:106860004146CE0031492B008E19220034687568EC
:106870002000290001F0F6FE009001910098019996
:1068800022002B0003F086F802B004BC9046F0BD55
:10689000332A08DD8023DB009A42F5D102000B0089
:1068A00001F0E0FEF0E7224A94460122634452429E
:1068B000DA400242E8D052080242D1D0944380220A
:1068C000D2051A411443CBE74B005B080343DBD0EE
:1068D0000B031B0B1C436342234380244D0C2403F6
:1068E0001B0B23406D042B4319004346DA000F4B6A
:1068F0009B181C685D6802000B002000290001F055
:10690000B1FE009001910098019922002B0003F044
:1069100041F842464B005B08D60733431900B3E702
:1069200001FCFFFFFFFF0F00EEFBFFFF20CB00008D
:10693000EDFBFFFFF8B5274A4B005B0D9A180C00E2
:106940000700132A10DC002A36DB234B13410B42CD
:106950003AD0802424031441002064189C4306008C
:10696000250030002900F8BD332A0EDD8023060003
:10697000DB000D009A42F4D102000B003800210028
:1069800001F070FE06000D00EBE7144D0600AC466A
:10699000012563446D42DD40AC4663460D00034271
:1069A000DFD033239A1A323B93401818874200D91C
:1069B0004C1C63469843D2E7C90FCC070020531CF8
:1069C000CDD1074B1C43CAE706000D000028C0D1FB
:1069D000C7E7C04601FCFFFFFFFF0F00EDFBFFFF15
:1069E0000000F03F30B5214A4B0087B05B0893426E
:1069F0001EDD1F4A934205DD02000B0002F0CAFFB4
:106A000007B030BD02AA00F095F803231840049A9D
:106A1000059B012813D002281DD0002814D002980D
:106A2000039900F06FFB80231B069C466144E7E757
:106A3000002300220093002301F0DEF8E0E7029833
:106A4000039900F05FFBDBE70124029803990094AF
:106A500001F0D2F8D4E7012402980399009401F0E0
:106A6000CBF880231B069C466144C9E7FB21E93F24
:106A7000FFFFEF7FF0B54746CE4680B58DB00400EE
:106A80000D0000F067FA294B06001B780F005BB27F
:106A90009846013310D022002B002000290003F07B
:106AA000C1FA8146002807D10022002320002900D6
:106AB00001F00AFC002806D1300039000DB00CBCF2
:106AC00090469946F0BD01230293194B0694079511
:106AD00003934B460A93434604940595002B15D027
:106AE000002300221900100002F0D8F84346089055
:106AF0000991022B0ED103F0AFFB212303600A9B07
:106B00000193002B0CD1089E099FD5E70023002498
:106B10000893099402A801F0C1F90028EFD1EAE72F
:106B200003F09AFB0A9B01930360ECE760000020EE
:106B300030CB0000F0B54E464546DE465746E0B540
:106B4000E14B4C008FB09046894664089C4200DCC3
:106B500087E0DE4B9C4222DCDD4A002900DC92E02B
:106B6000DC4B02F017FFDB4B06000F009C4200D10C
:106B70007EE1D94AD94B02F00DFF02000B004146DD
:106B800030000A604B60390002F004FFD34BD24A58
:106B900002F000FF434601259860D9606BE0D04BBE
:106BA0009C4200DC8FE0CF4B9C4200DD55E1CE4A99
:106BB000231592469A4451460905631A19001D008F
:106BC000040003F04BFA03F07FFA02000B002000F0
:106BD00029000892099302F0DDFE0022C34B02F067
:106BE00067FC0F00060003F039FA03F06DFA0400A9
:106BF0000D0002000B00300039000A940B9502F0E2
:106C0000C9FE0022B94B02F053FC002200230C9075
:106C10000D9101F053FB002800D192E100230022E6
:106C20002000290001F04AFB434243410133B04AAE
:106C300041460192022208A80092524600F07CFBD5
:106C40004B460500002B16DA802243461206944676
:106C500042465B68454263445360D3686344D360F3
:106C600009E00B00020041460A604B60002200234D
:106C700000258A60CB6028000FB03CBC9046994646
:106C8000A246AB46F0BD934B01F0ECFC914B0600E5
:106C90000F009C4200D13DE18F4A904B01F0E2FC95
:106CA00002000B00414630000A604B60390002F0E0
:106CB00071FE894A894B01F0D5FC012543466D429E
:106CC0009860D960D7E701F049F88A4A8A4B0600F4
:106CD0000F0002F0EDFB0022884B01F0C3FC03F033
:106CE000BDF9050003F0F0F9794A7A4B049005915B
:106CF00002F0DEFB02000B003000390002F04AFE19
:106D0000754A06000F0004980599744B02F0D0FBF9
:106D1000029003911F2D00DCC7E0029A039B300014
:106D2000390002F037FE83468A4653465B0024153D
:106D30005B0DE31A102B6CDD04980599D322674B89
:106D4000520502F0B5FB02000B0030003900029240
:106D5000039302F01FFE0A00010013000691079240
:106D600002003900300002F015FE029A039B02F087
:106D700011FE06000F0004980599614A614B02F06C
:106D800097FB32003B0002F005FE069E079F0B00BA
:106D90000200390030000292039302F0FBFD4B0029
:106DA0005B0D83468A46E41A312C32DD049805993E
:106DB000B822544B920502F07BFB03000C0002004A
:106DC000029303940B000698079902F0E3FD02007A
:106DD0000B0006000F000698079902F0DBFD029AEF
:106DE000039B02F0D7FD484A02900391049805994D
:106DF000464B02F05DFB029A039B02F0CBFD0200C2
:106E00000B00300039000292039302F0C3FD834669
:106E10008A465A465346414630000A604B60390064
:106E200002F0B8FD029A039B02F0B4FD44460B0049
:106E30000200A260E3604B46002B00DB1BE75B46D1
:106E4000236080231B065344636080231B069C46FB
:106E50006144A060E1606D420DE70B00020002F0AA
:106E600099FD434600259860D9601860596002E793
:106E7000D3221A4B520502F08DFD214A214B0D0001
:106E8000040002F087FD02000B00414620000A606A
:106E90004B60290002F07EFD1A4B194A02F07AFD80
:106EA000434601259860D960E5E602000B003000FA
:106EB000390002F06FFD6B1E154A9B009B588346FC
:106EC0008A46A342A5D130E7FB21E93F7BD90240A6
:106ED00000004054FB21F93F3163621A61B4D03D98
:106EE000FB213941FFFFEF7FEAFBFFFF000070410C
:106EF000B8CB000083C8C96D305FE43F0000E03FBD
:106F00007370032E8A19A33BC14920259A837B39CC
:106F100038CB0000D3220C4B520501F0A3FB0B4AE7
:106F20000B4B04000D0001F09DFB02000B004146DD
:106F300020000A604B60290002F02CFD034A044B3C
:106F4000B9E6032373E6C04661B4D03D7370032EE7
:106F50008A19A33BF8B54746CE46674B80B50A0071
:106F60000F00190005003940994200D19BE0040050
:106F70000100002F69DD3F1500D1B4E05F4B120323
:106F80009C468023120B5B0313435B00CA0F6744CC
:106F90009B184A00F80703D5D20F5B009B188A00A4
:106FA00079108C46002180201624894680030D1814
:106FB0009D4202DC29185B1B8144D50F5B00013C1C
:106FC0005B1952004008002CF1D10020804680203F
:106FD00020250027000609E08B425CD0D40F5B001F
:106FE000013DE31852004008002D16D0C4198B4211
:106FF000F2DD27180E00002C49DB5B1AA242894102
:1070000049425B1A121BD40F5B00013D80443100E2
:10701000E31852004008002DE8D113434ED14346F7
:107020005B0837494A468846494652104244C907D8
:1070300002D5802109060B4361460F05BD181800D3
:1070400029000CBC90469946F8BD7B005B080343C1
:107050003900002BF5D0002F3CD1E30A153A640526
:10706000002BFAD08020400303423FD1002700E0EC
:107070000F005B00791C0342FAD0250020208D40D0
:10708000401A2900D71B2200C2401A4376E7FE436C
:10709000F60F8E19B1E79442A0D82718002CF6DB22
:1070A0001E000023AEE702003B002800390002F07A
:1070B000FFF92A003B0001F0D5FAC2E7434601334D
:1070C00003D0434601335B08ABE701239846002316
:1070D000C144A6E73B00020002F05CFC02000B008A
:1070E00001F0DCFDADE713000022BBE70127210022
:1070F00020207F42C6E7C0460000F07F01FCFFFF72
:107100000000E03FF0B54746CE4680B587B000921C
:107110000193754B4F00814688467F089F4263DC90
:1071200002F09CFF002800D1D4E04A46434648467E
:10713000414602F0BDF904000D006C4A6C4B02F0B0
:10714000B7F96C4A6C4B01F08DFA22002B0002F06B
:10715000AFF96A4A6A4B02F01DFC22002B0002F0D4
:10716000A7F9684A684B01F07DFA22002B0002F073
:107170009FF9664A664B02F00DFC22002B0002F0DC
:1071800097F9644A644B01F06DFA22002B0002F07B
:107190008FF9029003910022604B2000290002F039
:1071A00087F9029A039B06000F002000290002F0D5
:1071B0007FF9009A019B04000D004846414602F009
:1071C00077F902000B002000290002F0E3FB020027
:1071D0000B003000390002F0DDFB02000B00002044
:1071E0004F4902F0D7FB70E002000B0002F060F99B
:1071F00004000D003D4A3E4B02F05AF93D4A3E4B19
:1072000001F030FA22002B0002F052F93B4A3C4BCD
:1072100002F0C0FB22002B0002F04AF9394A3A4B37
:1072200001F020FA22002B0002F042F9374A384BD5
:1072300002F0B0FB22002B0002F03AF9354A364B3F
:1072400001F010FA2B00220002F032F9354B0290C7
:1072500003919F429FDD344B00229F423DDC334926
:1072600000207B182E4916001F0002F093FB0490AB
:1072700005910022294B2000290002F019F9320063
:107280003B0002F087FB029A039B06000F002000E0
:10729000290002F00DF9009A019B04000D004846F8
:1072A000414602F005F902000B002000290002F01F
:1072B00071FB02000B003000390002F06BFB020092
:1072C0000B000498059902F065FB07B00CBC9046D2
:1072D0009946F0BD00201249F7E7154B00260492AD
:1072E0000593144FC5E7C046FFFF3F3ED43888BE24
:1072F000E9FAA8BDC4B1B4BD9EEE213EAD529C805A
:107300004F7E923E9015CB19A001FA3E7751C116DF
:107310006CC1563F4C5555555555A53F0000E03FB3
:107320000000F03F3233D33F0000E93F0000E0FFB0
:107330000000E73F0000D23FF0B5DE464E4645462E
:107340005746E0B5DC4CA5440D9114001900A49AF1
:107350000993DA4B9200D6584D1E03901821E01E77
:107360000696029500F0A0FEC3430100DB1719400A
:107370004B1C9A009B1ADB001B190B9105934C1BAD
:10738000771918D4A59BA5009C463F1922AE6544E9
:10739000013707E0286802F097FE013403C6043580
:1073A000BC4208D0002CF5DA00200021013403C6CD
:1073B0000435BC42F6D1069B002B01DA00F0FDFB40
:1073C000069B03990133DB009A46099BDA00944639
:1073D00000920022914672AA0492B94A61449346EF
:1073E00088469AAB63449B44029B002B00DABCE1C5
:1073F0005D4600260027039C4D442A686B6803CC39
:1074000002F056F802000B003000390001F02AF9B2
:10741000083D06000F004445EFD1049B4B441E601D
:107420005F6008239C46E144D145DDD10EA80421CC
:107430008446494261448C46069A93009C446146C6
:1074400084460A910399083B63448C460C93009B45
:10745000009263449B46009A0498D10003008C4636
:10746000634408911E685F68002A33DD95498046B1
:107470008C466244D300984470AB9A460EAB994652
:107480000022914B3000390002F012F802F0E6FDC4
:1074900002F01AFE00228D4B04000D0002F008F8E5
:1074A00002000B003000390002F074FA02F0D6FD41
:1074B0004B4601C39946434620001A685B68290081
:1074C00001F0D0F808235B429C46E04406000F0020
:1074D000D045D5D1059B30001A003900984600F000
:1074E000DFFCFF2300229B0504000D0001F0E0FFFC
:1074F00000F038FC0022764B01F0DAFF02000B00AE
:107500002000290002F046FA0D00040002F0A6FD5A
:10751000814602F0D9FD02000B002000290002F094
:1075200039FA060040460F00002800DCEEE0009B20
:1075300018215A1E92000EAB9B58091A1D000D41CE
:10754000A9448D405D1B0EAB9D5017231B1A1D4196
:10755000002D2DDD01239C46009BE144002B00DC27
:107560001CE20E9C0123002C00D0B5E0009A012AF9
:1075700009D099000EAA54580133002C00D0ACE079
:10758000009A9A42F5D1059B002B0EDD012B00D10C
:10759000A8E1022B09D1009B0EA95A1E92000EAB46
:1075A0009B5807939B029B0A8B50022D00D1C1E090
:1075B000002300223000390000F080FE009B0028EC
:1075C00000D194E2069A591E8A4210DC414A0A9878
:1075D00094460EAA6344944600229B0063441C68B0
:1075E000043B22438342FAD1002A00D0C0E0069B2C
:1075F0000EAA013B9B00D358002B00D0B3E0012220
:107600000C9B043B596801320029FAD0009B9C4630
:107610006244110007921A0001338B4246DC0B983A
:1076200063468046A59C4344A046099C9B00A14616
:107630004A449844D30022AA9146049A9944944615
:10764000089BA59A63448446614494469A468B00FD
:10765000634400934346586802F036FD4B46186079
:107660005960029B002B24DB4D46039C002600271B
:1076700001E0286869680CCC01F01AFF02000B00D9
:107680003000390000F0EEFF083D06000F005C45B9
:10769000EFD153469E60DF6004239C460433E044F0
:1076A0009C46009BE144E2449845D3D1079B00935C
:1076B000D1E600260027ECE794FDFFFF00CD000097
:1076C00018FEFFFFFFFFFF1F0000703E000070412B
:1076D00000002040FFFFFF3F002180225204141BC6
:1076E0000EAA5450009999420EDD0EA884469B00C4
:1076F0000EAA8900D25861446344CF4800E01A685A
:10770000821A04C38B42FAD101243CE7059B002B6B
:1077100006D1009B0EAA013B9B00D558ED1517E73B
:107720000022C64B300000F0EDFD002800D024E11F
:1077300000253DE732003B000020C14902F02AF954
:1077400006000F00002C00D132E7059A0020BC494A
:1077500000F0A6FB02000B003000390002F01AF91D
:1077600006000F0024E7012250E70026002754E618
:107770004B46059A079388468B000EA9CB58183ABA
:1077800008950592002B0DD18C464146AD4B4344E4
:107790009B006344043B58680139183A0028F9D02B
:1077A00088460592059A0020A54900F079FB4346DA
:1077B00004000D00002B00DA05E29E000EAB9C4693
:1077C0004346DB0066449C46059370AB9946049F94
:1077D00067440097306802F077FC22002B0001F02C
:1077E00067FE002238607960974B2000290001F085
:1077F0005FFE083F04000D00043EB945EAD14AABE4
:1078000003939B4600239A46069B4246994643466D
:107810000132029204934B46002B00DAAAE080204A
:107820008A4B009D9846C005894900260027002400
:1078300008E008239C460835E044544511DC4346E3
:10784000186859682A686B6801F032FE02000B0064
:107850003000390000F006FF013406000F00A1459A
:10786000E7DA5B46C0C39B4601239C46009BE2448B
:10787000083B0093029B9A45CDD1049B9846A49B5C
:10788000022B00DD8EE0002B37DC1FD1059B00278B
:107890001D00039B00249C461E006544083E2A6888
:1078A0006B683800210000F0DDFE083D07000C0089
:1078B000AE42F4D1089B002B03D080231B069C46CC
:1078C00064443A0023000D990A604B600720079B2F
:1078D00018409B239B009D443CBC90469946A24681
:1078E000AB46F0BD009B0EA95A1E92000EAB9B58F2
:1078F00007935B025B0A8B5057E64346002B00DA86
:1079000070E100200021DB004AAAD61848AF326897
:107910007368083E00F0A6FEB742F8D1089B002B22
:1079200000D025E10B0002004A984B990D9C226083
:10793000636002F02FF8434607000C00002B13DDB4
:1079400001254CAEB14638002E0021004C460136D0
:107950000CCC00F087FEA146B045F7DA089B070083
:107960000C00002B00D015E13A0023000D998A602D
:10797000CB60ABE70026002773E701239C46009B02
:10798000E1440225002B00DDEBE532003B00002046
:107990002B4901F0FFFF06000F0009E60024F2E585
:1079A0004AAB0393A49B032B00D08FE74346002BE5
:1079B00000DC14E1039ADB009B46130091465B4414
:1079C0001E685F68234B43440293DB00994448AB35
:1079D0009A464B465C681B681800210032003B0049
:1079E0000090019100F03EFE04000D0002000B002B
:1079F0000098019901F0CEFF3B00320000F032FE0A
:107A00004B469860D9601C605D6008235B429C46D1
:107A1000E14426002F00CA45DBD14346012B00DCA0
:107A2000E3E0039A13005B441E685F68029BDB007F
:107A300099464A44904610E0FFFFFF000000E03FF7
:107A40000000F03FFFFFFF3F0000703EC0CC000091
:107A5000FB21F93FFFFFFF1F984643465C681B6808
:107A60001800210032003B000090019100F0FAFD67
:107A700004000D0002000B000098019901F08AFF3C
:107A800032003B0000F0EEFD4346039A9860D96057
:107A90001C605D60083B26002F009A42DCD14D46F9
:107AA0009446002600244746083565442A686B68DA
:107AB0003000210000F0D6FD083D06000C00AF426A
:107AC000F4D1039B4A9F5D689968D868089B002B96
:107AD00065D08022120694460D9B65446044644440
:107AE0001F605D609960D8601E615C61EEE69A4639
:107AF0004B460793059B30005A423900089500F029
:107B0000CFF900223A4B06000F0000F0FBFB0028E3
:107B100024D0384B00223000390001F0C9FC02F0BB
:107B20009DFA52460400950002F0CEFA0022304B36
:107B300001F0BEFC02000B003000390001F02AFF0A
:107B400002F08CFA0EAA50510122059B52441833C0
:107B50009046059393000EAAD45023E65346300076
:107B600039009C0002F07AFA0EAB1851D04619E6A3
:107B700080230D9A1B06CB18106053600B00020087
:107B80004A984B9901F006FF434607000C00002B72
:107B900000DDD5E680231B069C466444E4E62B000A
:107BA0003A000D9D2A606B600A000300AA60EB603A
:107BB000320023002A616B6188E6099BDB00009399
:107BC00072AB049332E4A49B022B00DDE8E6002BA9
:107BD00000DD92E600D079E6002700246AE6002660
:107BE00000246EE70020002198E60026340068E7B4
:107BF000000070410000703EF0B5CE46474680B5AB
:107C000087B000920193474A4B00814688465B0843
:107C1000934207DC4146484602F020FA4146031EE3
:107C2000484666D04A4643464846414601F040FC35
:107C300004000D0002000B004846414601F038FCEC
:107C4000394A3A4B06000F002000290001F030FCB1
:107C5000374A384B01F09EFE22002B0001F028FC31
:107C6000354A364B00F0FEFC22002B0001F020FCD0
:107C7000334A344B01F08EFE22002B0001F018FC39
:107C8000314B324A00F0EEFC0E9B02900391002B28
:107C900034D00098019900222D4B01F009FC029A82
:107CA000039B049005913000390001F001FC0200B3
:107CB0000B000498059901F06DFE22002B0001F0E5
:107CC000F7FB009A019B01F065FE224A04000D00BB
:107CD000214B3000390001F0EBFB02000B002000CB
:107CE000290000F0BFFC02000B004846414601F0AD
:107CF00051FE07B00CBC90469946F0BD02000B0047
:107D00002000290001F0D4FB124A134B01F042FE7F
:107D100032003B0001F0CCFB4A46434600F0A2FC97
:107D2000E7E7C046FFFF3F3E7CD5CF5A3AD9E53D55
:107D3000EB9C2B8AE6E55A3E7DFEB157E31DC73E1C
:107D4000D561C119A0012A3F1111813FA6F8101178
:107D50000000E03F495555555555C53F49004B0872
:107D600019007047474AF0B54F4691464B005B0DEE
:107D700099444646D6464A46C0B505000C000E005A
:107D800088460700132A27DC002A4BDB3E4B1341B1
:107D90009A460B0052461340034318D03B4A3C4BD3
:107DA0002800210000F05EFC0022002300F0A0FA71
:107DB000002847D0002C04DA80234A465B03134195
:107DC00098444646534600279E43380031001CBC69
:107DD00090469946A246F0BD332A08DD8023DB0099
:107DE0009945F4D102000B0000F03CFCEFE7294A72
:107DF0009446012263445242DA4092460242E6D05F
:107E0000224A234B2800210000F02CFC00220023F2
:107E100000F06EFA002815D0002C1EDB53464646B3
:107E20009F430FE0194A1A4B2800210000F01AFC6A
:107E30000022002300F05CFA002803D0002C04DBB1
:107E40000027002638003100C1E76400640825439C
:107E50000027002DF6D0104EF4E74B46142B0BD024
:107E60003422D21A012393405D19BD4208D2012366
:107E70009C462F00E044D1E7133B9C46E044CDE70D
:107E80002F00CBE701FCFFFFFFFF0F009C75008870
:107E90003CE4377EEDFBFFFF0000F0BF00207047A1
:107EA0004B0070B55B0D14000A00002B1AD14B007B
:107EB0005B08034315D0234B002201F0F9FA224B53
:107EC0009C422DDB0A004B005B0D363B1F4DE31837
:107ED000AB422ADC002B0DDD1D4C1B0522401A4352
:107EE000110070BD1B4DAB42F0D102000B0000F041
:107EF000B9FBF6E71D00353519DA174B02009C4235
:107F000009DD0B001548164900F032F8134A144BEE
:107F100001F0CEFAE5E70B001248134900F028F80B
:107F2000104A114B01F0C4FADBE70200E9E7084C04
:107F3000363322401B051343190000220B4B01F07E
:107F4000B7FACEE700005043B03CFFFFFE07000049
:107F5000FFFF0F80FF07000050C300009C750088E2
:107F60003CE4377E59F3F8C21F6EA5010000903C37
:107F700030B54A00DB0FDB0752081A43110030BD51
:107F800002B4714649084900095C49008E4402BCAC
:107F90007047C046002243088B4274D303098B42CA
:107FA0005FD3030A8B4244D3030B8B4228D3030CC9
:107FB0008B420DD3FF22090212BA030C8B4202D36B
:107FC0001212090265D0030B8B4219D300E0090A93
:107FD000C30B8B4201D3CB03C01A5241830B8B429C
:107FE00001D38B03C01A5241430B8B4201D34B0385
:107FF000C01A5241030B8B4201D30B03C01A5241EA
:10800000C30A8B4201D3CB02C01A5241830A8B426E
:1080100001D38B02C01A5241430A8B4201D34B0257
:10802000C01A5241030A8B4201D30B02C01A5241BB
:10803000CDD2C3098B4201D3CB01C01A524183096F
:108040008B4201D38B01C01A524143098B4201D3A9
:108050004B01C01A524103098B4201D30B01C01AD4
:108060005241C3088B4201D3CB00C01A524183084E
:108070008B4201D38B00C01A524143088B4201D37B
:108080004B00C01A5241411A00D2014652411046DB
:108090007047FFE701B5002000F0F0F802BDC046D0
:1080A0000029F7D076E7704703460B437FD40022C0
:1080B00043088B4274D303098B425FD3030A8B427C
:1080C00044D3030B8B4228D3030C8B420DD3FF22E6
:1080D000090212BA030C8B4202D31212090265D0B4
:1080E000030B8B4219D300E0090AC30B8B4201D367
:1080F000CB03C01A5241830B8B4201D38B03C01AAE
:108100005241430B8B4201D34B03C01A5241030B24
:108110008B4201D30B03C01A5241C30A8B4201D3D5
:10812000CB02C01A5241830A8B4201D38B02C01A80
:108130005241430A8B4201D34B02C01A5241030AF7
:108140008B4201D30B02C01A5241CDD2C3098B42DC
:1081500001D3CB01C01A524183098B4201D38B0159
:10816000C01A524143098B4201D34B01C01A5241FC
:1081700003098B4201D30B01C01A5241C3088B4241
:1081800001D3CB00C01A524183088B4201D38B002C
:10819000C01A524143088B4201D34B00C01A5241CE
:1081A000411A00D201465241104670475DE0CA0FA5
:1081B00000D04942031000D34042534000229C4665
:1081C00003098B422DD3030A8B4212D3FC2289016F
:1081D00012BA030A8B420CD3890192118B4208D345
:1081E000890192118B4204D389013AD0921100E0A7
:1081F0008909C3098B4201D3CB01C01A52418309BB
:108200008B4201D38B01C01A524143098B4201D3E7
:108210004B01C01A524103098B4201D30B01C01A12
:108220005241C3088B4201D3CB00C01A524183088C
:108230008B4201D38B00C01A5241D9D243088B42E2
:1082400001D34B00C01A5241411A00D20146634685
:1082500052415B10104601D34042002B00D54942E9
:10826000704763465B1000D3404201B5002000F028
:1082700005F802BD0029F8D016E770477047C046E0
:10828000D0400B1C1141203A03D49C4613411843A3
:1082900063465242934018437047C0468446101CC0
:1082A00062468C46191C634600E0C0461FB501F0CB
:1082B00097F8002801D40021C8421FBD10B500F076
:1082C000EFFF4042013010BD10B501F089F80028E1
:1082D00001DB002010BD012010BDC04610B501F02B
:1082E0007FF8002801DD002010BD012010BDC04630
:1082F00010B501F011F8002801DC002010BD0120AC
:1083000010BDC04610B501F007F8002801DA0020C2
:1083100010BD012010BDC046F0B5CE46474615043D
:108320002D0C2E0080B50704140C3F0C9946030C4D
:108330007E435D43674363437F19340CE4199C46D5
:10834000A54203D980235B029846C4444B4643436D
:108350005143250C36046544360C2404A4195B19DA
:10836000591820000CBC90469946F0BDF0B54E4619
:1083700057464546DE46E0B543025B0A450083B0FA
:108380000F1C99462D0EC60F002D57D0FF2D24D05F
:108390008020DB00C0041843002381469A469B4698
:1083A0007F3D7C027A00FB0F640A120E984623D0B0
:1083B000FF2A4BD0E30080240020E4047F3A1C43D2
:1083C000AD186B1C47460193534677403A000F2B7C
:1083D00048D87D499B00CB589F46002B00D085E0B4
:1083E00008339A46063B9B467C027A00FB0FFF252A
:1083F000640A120E9846DBD1002C00D090E0524661
:1084000001231A4392460120DBE74C4658461700E9
:10841000022824D0032800D1CFE000220023012825
:108420004DD15802D205400AFF071043384303B02C
:108430003CBC90469946A246AB46F0BD002B5BD1B2
:1084400004239A46033B00259B46AAE7FF35002CF0
:1084500060D1524602231A4392460220B1E7FF221E
:108460000023DEE74B461B0C9C464B462604360C8D
:10847000180461463300220C6446000C43434E430B
:108480005043544380191A0C1218964203D9802184
:1084900049028C4664441B041B0C1004C018830161
:1084A0005E1EB341800E1843130C1B199B0103433E
:1084B0001C00230179D5012362081C401443019A52
:1084C0007F32002A4DDD630704D00F232340042BA5
:1084D00000D00434230103D53C4B019A1C40803268
:1084E000FE2ABCDCA3015B0AD2B29AE70C239A46AF
:1084F000093BFF259B4654E7180001F071FE4A46F0
:10850000431F76259A4000236D4291462D1A9A46C4
:108510009B4646E7524603231A439246032050E700
:10852000200001F05DFE431F2D1A9C40763D002087
:1085300047E780230027DB03FF2272E7424666E716
:108540004C463200584662E780234A46DB031A4213
:1085500022D01C4220D123435B025B0A4746FF2204
:108560005FE701239A1A1B2A21DC23000199D340DB
:108570009E318C401A0023005C1EA34113435A070E
:1085800004D00F221A40042A00D004335A0111D417
:108590009B015B0A002244E780234A46DB03134326
:1085A0005B025B0A3700FF223BE7019587E7002269
:1085B000002336E70122002333E78023DB03234334
:1085C0005B025B0AFF222CE710CD0000FFFFFFF7E4
:1085D00070B500283DD0C317C5185D40C40F2800F2
:1085E00001F0FEFD9E22121A962A07DCD2B208285C
:1085F00033DD083885406802400A23E0992A0BDD04
:10860000052329001B1AD94003001B339D402B0072
:108610005D1EAB4119430D00052801DD431F9D4040
:108620002B000F490B406E0709D00F263540042D53
:1086300005D004335D0102D59F220B40121A9B0125
:10864000580AD2B24002D205400AE4071043204340
:1086500070BD002400220020F4E76802400AF1E720
:10866000FFFFFFFBF0B54F464646D6460C00090318
:10867000C0B5490A470F5E0039431F03DB0F9C4614
:1086800065007B0A570F1F436D0DE40F760DA14661
:10869000C000B846D200AB1B64457BD0002B5FDD29
:1086A000002E00D0A4E03E00164300D112E15E1E71
:1086B000002E00D09EE1871A4346B8428041012532
:1086C000C91A4042091A0B0200D431E149024E0A8C
:1086D000002E00D16EE1300001F082FD0300083B66
:1086E0001F2B00DD61E120223900D21A9E40D140CB
:1086F0009F400E439D4200DD51E15D1B6B1C1F2B13
:1087000000DD7CE12021C91A3D0030008F40884007
:10871000DD40791E8F41310007222843D9400025D2
:1087200007433A40002A09D00F233B40042B05D0D1
:108730003B1DBB42BF417F42C9191F000B0200D441
:1087400026E26A1CC64B55056D0D9A4200D106E122
:10875000C44AFF080A40530752023B43120B8EE003
:10876000002B00D0B8E06B1C5B055B0D012B00DC1F
:1087700030E1871A4346B842B641CB1A76429E1B77
:10878000330200D54CE13B003343A1D10022002449
:10879000002570E0002B00DCE5E0002E00D183E036
:1087A000AF4EB54260D0802636043743B846382BEA
:1087B00000DC3EE1434613431F007A1E97413F18F9
:1087C00087428041404209180B0200D4B0E0A44B1C
:1087D00001359D4200D1C3E0A24A7B080A40012135
:1087E0000F401F435108D30707221F433A4099E720
:1087F0009B4EB54238D0802636043743B846382BD6
:1088000000DDDCE01F2B00DC30E11E004746203E8F
:10881000F740BC46202B04D04026F31A46469E4023
:108820003243170063467A1E97411F43CCE0002B6A
:1088300000D104E24346134300D159E14B07C0087D
:1088400018438023C9081B03194208D04546ED0888
:108850001D4204D14346D008590708432900420F5E
:10886000C9007F4D1143C0004B07CA087C49C008AE
:1088700003438D4268D012036D05120B6D0D00216C
:1088800012031800130B0A0D12051A43764B2D051F
:1088900013402B435B00E4075B08234319001CBC17
:1088A00090469946A246F0BD3E00164312D05E1E89
:1088B000002E00D000E187188742804141444042A9
:1088C000091801250B0233D5022585E764463300DC
:1088D000414610001D00C7E7002D00D0DAE00C0073
:1088E0000443F3D05C1C00D19FE15D4CA64200D153
:1088F0002FE1DB43382B00DD66E11F2B00DD83E138
:1089000020240500E41A0F00DD40D940A040434672
:10891000A7405B1A441EA04198462F433843171ABC
:10892000BA42924143465242991A64463500CAE619
:1089300007223A40002A00D0F6E64B07CA08484909
:10894000FF083B438D4296D11900114300D19EE1AF
:10895000802109030A431203120B414D8FE71500D2
:10896000002200238BE7002B00D0C7E06B1C5F05C3
:108970007F0D012F00DCF1E0394DAB4200D1B9E0B1
:1089800085180A008542894142444942511807220C
:10899000CF076D082F4349083A401D00C2E6072261
:1089A0003049ED1A31403A40BCE63E002838864056
:1089B00000279FE6380001F013FC20308EE6434686
:1089C00013431F007A1E9741C71BB84280414042A3
:1089D000091A78E60E003B0006431343002D61D1CF
:1089E000002E00D0F4E0002B00D11BE164463900DA
:1089F000100039E71A4FBB427AD03300FFE630004F
:108A00001F3DE840202B03D04021CB1A9E40374326
:108A10007B1E9F41072207433A400021002589E73A
:108A2000171A4346BA42B641591A76428E1B64461B
:108A30004EE61F2B00DDADE020264746F61AB74074
:108A4000B9461700B246DF404E463E433700564611
:108A5000B240561EB24117434246DA408918AEE68C
:108A6000FF070000FFFF7FFFFFFF0F802026474624
:108A7000F61AB740B9461700B246DF404E463E43AD
:108A800037005646B240561EB24117434246DA40BE
:108A9000891A99E77F4CA6425BD0802424045B426C
:108AA000214327E7002E0CD1002B00D1CBE06446F8
:108AB00039001000774DD7E6764FBB4218D033000F
:108AC00075E6002B14D04B07C00818438023C90853
:108AD0001B03194207D0FC081C4204D17907D008B7
:108AE0000843E14621004C46420FC9001143C00033
:108AF000684DB9E61D0000220023C0E6002D5BD1C1
:108B00000D00054300D1E2E65D1C00D1B0E0614DEF
:108B1000AE421FD0DB43382B71DC1F2B00DD96E00B
:108B200020250F00ED1AAF40B9460700AA46DF40E6
:108B30004D463D432F005546A840D940451EA8410B
:108B400088440743BF18974292415142414435003F
:108B50003AE6644635004146100085E60B000343C3
:108B6000002D00D063E6002BF5D04346134300D11F
:108B70007AE687188742804107224144404209181B
:108B80003A400B0200D4D5E6434B01351940C9E504
:108B9000380069E61E004746203EF740BC46202BC1
:108BA00004D04026F31A46469E40324317006346DF
:108BB0007A1E97411F4302E6364DAE42CAD0802549
:108BC0002D045B422943A6E70843411E8841A6E6DF
:108BD000002B00D148E6871A4346B842B641CB1A6B
:108BE00076429E1B33024BD5171A4346BA42924136
:108BF000591A5242891A072264463A4092E50143C3
:108C00000F00791E8F419DE71C000F00203CE740BC
:108C1000202B03D04024E31A99400843411E884189
:108C200038437CE60022002425E6171A4346BA4260
:108C30009241591A5242891A6446350043E5414629
:108C40001000144D10E680220024120380E61D005F
:108C50000F00203DEF40BC46202B03D04025EB1AEF
:108C60009940084307006346781E87411F4369E720
:108C7000871897429B4141445B42C9183500A3E5E0
:108C80003B003343CED0072231003A4052E6002366
:108C90001A00F4E5FF070000FFFF7FFFF0B557461D
:108CA000DE464E464546E0B5834607000E034800C3
:108CB00085B092461C00360B400DCD0F002800D128
:108CC0009DE0954B984239D08023F6001B041E434B
:108CD000924A7B0F334399469446030063440093C2
:108CE00000230026FF00029323031B0B984663001A
:108CF000E40F52465B0D019400D1B3E086498B42EC
:108D000000D19EE04246D100802212040A4351461F
:108D1000490F11438B46814952468C460099634462
:108D2000CB1A0021D20000932B0063409A460F2EED
:108D300000D905E17A4BB6009B599F465B46334309
:108D4000994600D0B8E0022308260027009002933D
:108D5000CAE7CB463A0002990195019B9A4602293F
:108D600027D0032900D180E2012944D06D49009B1E
:108D70008C4663441C00002C38DD530700D013E2FE
:108D8000D2085B46DB0109D55946674B19408B4633
:108D90008021C9008C46009B63441C00634B9C42AD
:108DA00007DC5B4664055F075B0217431B0B620D24
:108DB00002E000230027584A00211B031C0B0B0D67
:108DC0001B05234314055A4A380013401C435346DD
:108DD0006400DB0764081C43210005B03CBC9046DE
:108DE0009946A246AB46F0BD0122524201231B1B0D
:108DF000382B00DCADE1002200230027DCE75B46D6
:108E0000334399465ED0002E00D18AE1300001F054
:108E1000E7F903000B3B1C2B00DD7BE11D22D31A7D
:108E20005A460100DA4008398E4013005F4633434A
:108E300099468F403F4B00261B1A00930023029354
:108E400052E7414653460B433B499B468C46009BA9
:108E5000634400935B46002B3BD1022300221E4358
:108E6000022161E7434613439B4637D04346002B1C
:108E700000D162E1404601F0B3F903000B3B1C2B2B
:108E800000DD53E102004146083A914088461D2129
:108E9000CB1A5146D9400B0041460B439B465346E3
:108EA00093401A00009B25499C46604403008C4671
:108EB00063440093002137E70323B14600900C265A
:108EC000029311E700230093013304260027029345
:108ED0000AE70323C3461E43032125E701331E434C
:108EE0000022012120E700239A46802300271B034C
:108EF000094A61E7802349461B03194200D1E2E099
:108F00005946194200D0DEE00B431B0317001B0B30
:108F1000A246014A50E7C046FF07000001FCFFFFE0
:108F200050CD0000FF030000FFFFFFFEFE07000022
:108F3000FFFF0F800DFCFFFF01F8FFFFF3030000B0
:108F4000D94500D9CBE000D1C6E03C004846002717
:108F5000009B013B00935B46160E1B021E4313024F
:108F6000984633041B0C9946310C0191FFF798F891
:108F70004A4642430B04210C050019438A4207D993
:108F80008919013D8E4203D88A4201D9851E89196B
:108F9000881A0199FFF784F809048C464A4621048F
:108FA00064464243090C030021438A4204D98919CB
:108FB000013B8E4200D8F1E02D041D43AB464346F1
:108FC000891A4246280C12041D0C5B46140C220020
:108FD0001B041B0C5A4303946B43444302956843A0
:108FE0001B19150CEB189C4203D980246402A4467B
:108FF00060441C0C15041B042D0C20185D198142C3
:1090000077D373D00C1AA24A7D1BAF42BF4194465E
:10901000009B7F426344E01B1C00864200D1DBE0E2
:109020000199FFF73DF84A4642430B04290C07001B
:1090300019438A4207D98919013F8E4203D88A42CF
:1090400001D9871E8919881A0199FFF729F809049F
:109050004A46894629044D464243090C03002943E8
:109060008A4207D98919013B8E4203D88A4201D925
:10907000831E89193F04891A3A00039F1A43380056
:1090800013041B0C584381460298150C6F4343434D
:1090900045434846000C8446DB1963449F4203D98C
:1090A000802040028446654448461F0C00041B048F
:1090B000000C7D191818A94200D284E000D17FE08D
:1090C00001231A4357E680234A461B0313431B031D
:1090D0001B0BAA466F4A6FE6BA4200D935E74B46EA
:1090E000DC0758087B081C43FF0734E70024AF4225
:1090F00089D247444745A4415B466442A419641899
:10910000013BA6421ED2A0426DD800D1B6E0241A7F
:109110009B4678E703005A46283B9A400027914631
:1091200088E6584601F05CF8203072E603005246AB
:10913000283B9A4093460022B4E6504601F050F88E
:1091400020309AE6A642E2D1B845DCD9341A9B46D3
:1091500059E71F2B65DC504C0099A4465C466144DE
:1091600008008C4011008240D940501E82410C43BF
:1091700014435A46DA401300620709D00F222240F6
:10918000042A05D02200141D9442894149425B18EB
:109190001A0262D50122002300270DE68A4200D878
:1091A0000AE7831E891907E70F231340042B00D118
:1091B000E6E5171D9742924153429B44FA08E0E5C9
:1091C000002800D1D7E57118531EB14227D3A94218
:1091D00015D358D01A0073E7002B00DC04E60123F6
:1091E00000229B44CDE502234744474589415B4229
:1091F0009C46494289190C19E344241A03E7434663
:109200005F0047459B41B8465B429E19023A891967
:10921000A94200D054E7404500D051E7ABE51A0021
:10922000F6E71F215F4649420C1BE740202B07D081
:109230001A49009B8C46634418005B4683401A43DE
:10924000501E82413A4307270023174009D00F21BF
:10925000002311401400042995D122005F075B020E
:109260001B0BD20817430022A6E5802359461B0397
:109270000B431B0317001B0B064A9DE5BD42B2D8EA
:109280009B460024BFE68045B9D31A00C3E7C04619
:10929000FF030000FF0700001E0400003E04000062
:1092A000F0B54F464646D6468446C0B58046194E70
:1092B00018030F034D00000B5C0082463F0B6D0D41
:1092C000C90F9146640DDB0F0120B5420AD0B442AC
:1092D00003D0A54201D157450CD01CBC90469946FD
:1092E000A246F0BD66463E43F7D1AC42F5D15446A6
:1092F0001443F2D10120C845EFD1994207D0002D87
:10930000EBD163461F433800471EB841E5E7002014
:10931000E3E7C046FF070000F0B54F464646D64695
:109320004D00C0B50E03C90F8A462C491F035C00CF
:109330008046360B6D0D91463F0B640DDB0F8D4261
:109340001ED08C4216D0002D1ED130438446002CF6
:1093500001D13A4323D06246002A1AD09A4529D037
:10936000514602200139084001381CBC90469946FC
:10937000A246F0BD39001143E5D002204042F4E797
:109380003043FAD1AC420FD0002C0FD13A43E7D092
:109390000CE00122013B934318000130E5E76346EE
:1093A0000020002BE1D0DBE73A43E6D19A45D7D144
:1093B000A542D5DCA54205DBBE42D1D808D00020AD
:1093C000BE42D2D250460123013898430130CCE747
:1093D000C845C5D80020C845F4D3C6E7FF0700003C
:1093E000F0B54F464646D6464D00C0B50E03C90FF0
:1093F0008A462E491F035C008046360B6D0D914650
:109400003F0B640DDB0F8D4218D08C4211D0002D24
:1094100018D130438446002C1ED13A431CD16346F8
:109420000020002B30D0514602200139084001387D
:109430002AE039001143EAD0022025E03043FBD175
:10944000AC4226D0002C26D13A4324D151460220EA
:1094500001390840013817E06246002A0FD09A45CA
:10946000E1D1A54205DBBE42DDD819D00020BE42C5
:109470000AD25046012301389843013004E001220A
:10948000013B9343180001301CBC90469946A2460C
:10949000F0BD3A43D0D19A45C5D1A542C3DCE0E73F
:1094A000C845C0D80020C845E3D3EDE7FF0700005A
:1094B000F0B55746DE464E464546E0B583460600C3
:1094C0000F03480087B092461D003F0B400DCC0FA4
:1094D000002800D16FE0DE4B984238D08023FF0097
:1094E0001B041F43730F3B430193DA4B002799463C
:1094F00000239B46F60081442B0369001B0B524658
:109500009846490DED0F002900D185E0D04B9942D6
:1095100000D173E04346DA0080231B041343524614
:10952000CC48520F84461343524600206144D20077
:1095300089442100694000918C46012149448A46B2
:109540000F2F00D990E0C449BF00CF59BF465B46FA
:109550003B43019300D06AE102230827002681469D
:109560009B46C9E732005846019B6146009102289C
:1095700000D175E0032800D1FEE1012800D02CE1E4
:1095800000230027002600253F032A0D3F0BB34888
:1095900012053A4302401B051343009A5B00D107B2
:1095A0005B080B433000190007B03CBC904699465D
:1095B000A246AB46F0BD5B463B43019300D12FE191
:1095C000002F00D1A5E1380000F00AFE03000B3B9C
:1095D0001C2B00DD96E11D22D31A5A460100DA4009
:1095E0005E4608398F4013008E403B4301939C4BED
:1095F00000271B1A994600239B467DE741465346A8
:109600000B4393498C46E144002B00D01AE102221F
:109610000220174300228CE7134300D10DE143469B
:10962000002B00D181E1404600F0DAFD02000B3A48
:109630001C2A00DD72E10100434608398B40984640
:109640001D239A1A5346D3401A00434613435246E9
:109650008A404946081A824989468144002068E7C1
:109660007B4B002700268EE7140C1204120C11000D
:10967000370C3604350C794328008C462E006043A5
:109680006044834656432100300C80465846794357
:1096900040440291844506D98846802149028C467F
:1096A000E044414602913604010C360C00048B461E
:1096B00081191E0C1B041B0C0391190079438C4665
:1096C000280075436544A8465843050C4544774334
:1096D000A94203D9802149028C466744290C8C4653
:1096E00039000004000C2D042D186144AB44059191
:1096F0005946049101990F043F0C080C390051435D
:109700004243904602008C46090C8B4662437C43E0
:1097100044445C44A04503D9802149028846424420
:10972000210C884661460904090C8C4639005943CE
:10973000434370437E430F0CF6182404BE1964445F
:1097400042448C46B34203D980235B02984640448E
:10975000029B61469846049B370443449B46AB45B5
:10976000AD416B420D0405992D0C8C467F19674461
:10977000FD18A8465D462D19A542A44193466442B2
:10978000A446C344DC448F42BF4198459B41934566
:109790009241A445A4415B427F421F43360C524292
:1097A0006442BF192243BF18624638184302D20DE3
:1097B000039913436A020A43501E82416146ED0D2C
:1097C0002A434E023243D90100D4B3E001265008A7
:1097D00032400243DE0732435B08224C5444002CE3
:1097E00062DD510709D00F201040042805D0101D5C
:1097F0009042924152429B180200D90104D5802424
:109800001948E400034054441848844200DD27E727
:109810005E075B02D2081F0B630516435B0DB2E6C1
:10982000002399460133042700269B4664E6032360
:10983000019781460C279B465EE6012201201743D3
:10984000002276E6032303201F43434671E6C04609
:10985000FF07000001FCFFFF90CD0000FFFF0F801D
:109860000DFCFFFFFF030000FFFFFFFEFE070000EF
:109870000023802700933F030026434B83E6019B90
:109880003200A446584670E6AC466EE68027019941
:109890003F0339422DD03B422BD11F433F033F0BA7
:1098A00000951600384B6EE601252D1B382D00DD86
:1098B00066E61F2D40DC35481C00504416008240EF
:1098C0008440EE40501E824134431443EB40620713
:1098D00009D00F222240042A05D02200141D9442F0
:1098E000804140421B181A023ED501230027002662
:1098F00049E68027019B3F031F433F033F0B009432
:10990000214B40E603005A46283B9A40002601922C
:109910006DE6584600F064FC203057E603005246DE
:10992000283B9A401300002293E6504600F058FC72
:1099300020307BE6CA4650E71F201E004042041B31
:10994000E640202D03D0124C5444A3401A43501E2D
:109950008241324307260027164009D00F200023FA
:10996000104014000428B9D122005E075B021F0BCF
:10997000D2081643002306E680273F031F433F0318
:109980003F0B1600004BFEE5FF0700001E04000021
:109990003E040000F8B557464E464546DE460C00EC
:1099A0000903E0B5490A460F5F0031431E03DB0F90
:1099B000760A9B46530F3343C84E6500C000E40F40
:1099C000D2006D0DA24681467F0D9C469046B7425F
:1099D00000D1B9E05B46012673409B46EE1BA345D0
:1099E00000D183E0002E63DD002F00D0B1E063469C
:1099F000134300D123E1731E002B00D0BAE1861A75
:109A00006346B04280410125C91A4042091A0B023F
:109A100000D447E149024B0A98464346002B00D147
:109A200089E1404600F0DCFB0300083B1F2B00DD12
:109A30007CE120223000D21A4146D04099400200F9
:109A40009E400A439D4200DD6AE15D1B6B1C1F2B9B
:109A500000DD94E1202110003500C91A8E40DA4063
:109A60008840DD40711E8E411100072228430025E9
:109A700006433240002A09D00F233340042B05D07F
:109A8000331DB342B641764289191E000B0200D441
:109A90003DE26A1C914B55056D0D9A4200D119E1CA
:109AA0008F4AF6080A40570752023743120B9BE0D1
:109AB000002E00D0C5E06E1C7605760D012E00DC70
:109AC00048E16746861ACB1BB042BF417F42B84689
:109AD0001F004346FF1A3B00B8461B0200D55FE15A
:109AE00037439AD100220024002579E0002E00DCC3
:109AF000FAE0002F00D18DE0784B9D4267D08023A3
:109B000067461B041F43BC46382E00DC52E1634607
:109B100013435A1E93411E18864280414042091841
:109B20000B0200D4BEE06D4B01359D4200D1D2E066
:109B30006B4A73080A4001210E401E435108D307A7
:109B400007221E43324095E71E00164300D045E72A
:109B500040E7624B9D423AD0802367461B041F4377
:109B6000BC46382E00DDEBE01F2E00DC3AE133006E
:109B70006746203BDF403B00202E05D04027BF1B1F
:109B80006646BE40324390464646721E9641334377
:109B9000DAE0002B00D114E26346134300D168E100
:109BA00080234E07C008C9081B030643194208D08A
:109BB0006046C008184204D163460100D2085E071F
:109BC0001643F3009946C900720F444D11434B46AA
:109BD000DE08424B4F073743CA089D4200D16EE072
:109BE00012036D05120B6D0D00211203130B0A0DEC
:109BF00012051A433B4B2D0513402B435B00E40732
:109C00005B082343380019003CBC90469946A246A5
:109C1000AB46F8BD6346134311D0731E002B00D032
:109C200007E18618864280416144404209180125B7
:109C30000B0237D502257BE73E0061469146350091
:109C4000C5E75C46002D00D0E1E00B000343F3D0F4
:109C5000731C00D1ACE1214B9F4200D13AE1F343A8
:109C6000382B00DD6FE11F2B00DD8CE120250E007D
:109C7000ED1AAE40B0460600AA46DE4045463543E2
:109C80002E005546D940A8406346451EA8415B1AA0
:109C90009C463043161AB242924163465242991A88
:109CA0003D00B4E607223240002A00D0E4E60B4B28
:109CB000F6084F073743CA089D4200D090E73B00A3
:109CC000134300D1A6E180231B031A431203120B96
:109CD000024D89E715000022002785E7FF070000F5
:109CE000FFFF7FFFFFFF0F80002E00D0C7E06B1C3F
:109CF0005E05760D012E00DCF0E0C84DAB4200D1D0
:109D0000B9E085180A0085428941624449425118E8
:109D10000722CE076D082E43490832401D00A9E6F0
:109D2000BF49ED1A114007223240A3E6320028381D
:109D30008240002686E6300000F052FA203073E6BA
:109D4000634613435A1E9341C61AB04280414042B3
:109D5000091A5CE60E00674606431743002D5ED1E4
:109D6000002E00D0F3E0002F00D11EE15C466146DA
:109D700091462CE7A94FBE427BD01E00F1E61000B1
:109D80001F3DE840202B03D04021CB1A9A401643B8
:109D9000731E9E410722064332400021002583E7BF
:109DA000161A6346B2428041591A40420B1A98462D
:109DB0005C4632E61F2E00DDABE02027BB1B9A4637
:109DC00063465746BB40994613004F46F3401F4336
:109DD0003B005746BA40571EBA4113436246F24011
:109DE000891898E62027BB1B9A4663465746BB4016
:109DF000994613004F46F3401F433B005746BA4075
:109E0000571EBA4113436246F240891A9CE7834BBE
:109E10009F425FD080252D047342294320E7002E06
:109E20000CD1002F00D1D0E05C46614691467B4DBD
:109E3000CDE67A4FBE421CD01E0065E6002F18D03A
:109E4000C0084E0706438020C9080003014208D01D
:109E50006346DC08044204D12100DA46D2085E07DA
:109E60001643F300994601245346C900720F11436B
:109E70001C406A4DABE61D0000220027B4E6002D11
:109E800059D10B00034300D1D6E6731C00D1B2E0D8
:109E9000624B9F421ED0F343382B6FDC1F2B00DD3B
:109EA00097E020250E00ED1AAE40B0460600AA4607
:109EB000DE40454635432E005546A840D940451E54
:109EC000A8418C440643B6189642924151426144DF
:109ED0003D0025E63D006146914678E60B000343D0
:109EE000002D00D055E6002BF5D06346134300D17A
:109EF0006DE686188642804161444042091800227E
:109F00000B0200D4D0E6464B01351940B2E5B1460C
:109F10005DE633006746203BDF403B00202E05D046
:109F20004027BF1B6646BE40324390464646721EDF
:109F300096413343EFE5394B9F42CBD080252D042A
:109F400073422943A8E70843411E8841A2E6002F37
:109F500000D13CE66346861ACF1AB0429B415B4271
:109F6000FB1A98461B024ED5161A6346B24292411E
:109F7000591A5242891A5C4600227BE501430E00C1
:109F8000711E8E419FE71D000E00203DEE40B04641
:109F9000202B04D04025EB1A9940084381464846BF
:109FA0004346411E8841184374E60022002417E608
:109FB000161A6346B2429241591A5242891A3D001A
:109FC00025E561469146154D01E6802200241203E5
:109FD00079E61D000E00203DEE40B046202B04D057
:109FE0004025EB1A9940084381464E464346711E70
:109FF0008E411E4367E7861896429B4161445B424F
:10A00000C9183D008CE547463743CED0072241466C
:10A01000324049E600273A00E6E5C046FF07000067
:10A02000FFFF7FFF70B50C4E0D031C0349005B0062
:10A030002D0B490D240B5B0DB14208D006490020C1
:10A040008B4203D114432000441EA04170BD054340
:10A050000120002DFAD1F1E7FF07000030B5144DC3
:10A060000A034B00120B5B0DC90F0024AB4211DD3C
:10A07000104CA34210DC8024640322430E4CE41AEB
:10A080001F2C0CDD0D48C31ADA4013005C42002976
:10A0900000D11C00200030BD094BCC18FAE7094D57
:10A0A000E040AC4663449A4013000343EEE7C046E9
:10A0B000FE0300001D040000330400001304000030
:10A0C000FFFFFF7FEDFBFFFF70B500282DD0C3170A
:10A0D000C5185D40C40F280000F082F8154B1B1A0C
:10A0E0005B055B0D0A2815DD0B38854000222D032A
:10A0F0002D0B002110002D030A0D2D0B12052A43F4
:10A100000D4D1B052A4013435B00E4075B08234306
:10A11000190070BD02002900153291400A000B2180
:10A12000081AC5402D032D0BE3E70024002300256A
:10A130000022DEE71E040000FFFF0F804100090E31
:10A140004B1C70B5DBB24602750AC40F012B14DD3F
:10A15000E0239B006D07360BCB1800210A0D280069
:10A1600012051C4D32435B052A405B0813435B001C
:10A17000E4075B082343190070BD002914D1002DAA
:10A180001ED0280000F02CF80A281CDC0B232A0023
:10A190001B1ADA40030015339D400F4B12031B1AA4
:10A1A0005B05160B5B0DD8E7002D06D0320B802621
:10A1B00036036D071643094BCFE7084B0026CCE763
:10A1C00000230026C9E703002A000B3B9A40002524
:10A1D000E3E7C046FFFF0F8089030000FF07000090
:10A1E0001C2101231B04984201D3000C10391B0AC7
:10A1F000984201D3000A08391B09984201D300098B
:10A20000043902A2105C40187047C04604030202E1
:10A2100001010101000000000000000030B51C0039
:10A22000094B05001B6885B0D868084B002A01D18E
:10A23000074B1A000292019300912B00220005495E
:10A2400000F026F800F08EFD64000020D0CD000064
:10A25000EEBC0000DDCD0000014B18687047C04621
:10A2600064000020084B10B50400002B02D0002130
:10A2700000E000BF054B1868836A002B00D09847A8
:10A28000200001F045FBC046000000000CCE00009D
:10A290000EB403B5010003AB044804CB006801937E
:10A2A00000F076F802B008BC03B018476400002044
:10A2B00070B500260C4D0D4C641BA410A64209D1AC
:10A2C000002601F027FB0A4D0A4C641BA410A6428D
:10A2D00005D170BDB300EB5898470136EEE7B300E7
:10A2E000EB5898470136F2E7340200203402002090
:10A2F0003402002044020020002310B59A4200D10D
:10A3000010BDCC5CC4540133F8E710B5884202D9C3
:10A310008B18984203D3002307E08B5C8354013AE7
:10A32000FBD210BDCC5CC45401339A42FAD1F8E799
:10A3300003001218934200D1704719700133F9E7F6
:10A34000936810B5013B9360002B04DA9469A34233
:10A3500007DB0A2905D01368581C10601970080023
:10A3600010BD00F033FC0100F9E7F8B506000F005E
:10A370001400D518AC4201D1002007E021783A0042
:10A380003000FFF7DDFF0134431CF3D1F8BD0000BE
:10A39000F0B59FB002900F0016000593002805D07D
:10A3A00083690493002B01D100F0DCFD7B4B9F42BD
:10A3B0005BD1029B5F68BB891B0762D53B69002BA1
:10A3C0005FD0002306AC6361203363761033A3763D
:10A3D00035002B78002B01D0252B5CD1AB1B0493CF
:10A3E0000CD0320039000298FFF7BFFF431C00D1A8
:10A3F000C4E06269049B9446634463612B78002B3C
:10A4000000D1BBE0012200235242626002A9543213
:10A4100052186E1C2360E360A3601370A36531784B
:10A4200005225F4800F0BCFE751C002835D122686B
:10A43000D30604D5532302A95B18202119701307F2
:10A4400004D5532302A95B182B21197033782A2BCA
:10A450002CD0350000210A20E3682A786E1C303A9F
:10A46000092A64D900292ED026E04E4B9F4202D102
:10A47000029B9F689FE74C4B9F429CD1029BDF68E9
:10A4800099E73900029800F0F7FB002899D00120E5
:10A4900040421FB0F0BD01359BE7414B2268C01A16
:10A4A00001238340134323602E00B8E7059B191D49
:10A4B0001B680591002B01DB099304E05B42E3601C
:10A4C0000223134323602B782E2B0AD16B782A2B7F
:10A4D00035D1059B02351A1D1B680592002B2BDB1D
:10A4E0000793324E29780322300000F059FE0028ED
:10A4F00006D04023801B834022680135134323602C
:10A50000297806222A486E1C217600F049FE002890
:10A510003AD0284B002B25D10722059B07339343C4
:10A52000083305936369039A9B18636150E74343BB
:10A5300001219B18350090E701235B42D0E70023FF
:10A540000A201A000135636029786E1C3039092908
:10A5500003D9002BC5D00792C3E742430123521809
:10A560003500F1E705AB00933A00134B2100029848
:10A5700000E000BF0390039B0133D3D1BB895B068E
:10A5800000D584E70B9884E705AB00933A000A4BAB
:10A590002100029800F080F8ECE7C04664CE00008D
:10A5A00010CE000084CE000044CE000016CE000085
:10A5B0001ACE0000000000006BA30000F7B51500E4
:10A5C00001938A680B6900900C00934200DA130033
:10A5D00022002B6043321278002A01D001332B6015
:10A5E00023689B0602D52B6802332B60062723685D
:10A5F0001F4027D0230043331B785A1E9341226803
:10A60000920630D42200019943320098089EB04748
:10A61000431C25D0062320682A68E16803400025F2
:10A62000042B03D18D1AEB43DB171D40A36822696D
:10A63000934201DD9B1AED180027BD4220D1002076
:10A6400010E00137E3682A689B1ABB42D2DD220082
:10A650000123193201990098089EB047431CF0D19C
:10A6600001204042FEBD3020E11843310870210036
:10A670005A1C45310978A218433202331170C1E7E0
:10A68000220001231A3201990098089EB047431C0A
:10A69000E6D00137D1E70000F0B589B004920A0096
:10A6A00043320593039002920A7E0C000E9B6E2AA1
:10A6B00000D186E01FD8632A33D008D8002A00D101
:10A6C0008CE0582A4DD0250042352A7030E0642AAB
:10A6D00001D0692AF7D1196825680A1D280629D5ED
:10A6E00008681A60002803DA2D23029A404213708A
:10A6F0006B4E0A274FE0732A74D008D86F2A1FD0F8
:10A70000702AE0D1202209680A43226003E0752AFA
:10A7100016D0782AD7D12200782145321170614EA7
:10A7200022E025001A684235111D196013682B704C
:10A73000012365E008681A606906D3D500B2D1E745
:10A7400019682568081D186008682E0605D5544E3E
:10A7500008276F2A1BD00A2719E06D06F7D580B2AB
:10A76000F5E745314E4E0A7018682268011D0068F1
:10A770001960150621D5D30702D520231A4322607C
:10A780001027002803D1202322689A432260230047
:10A79000002243331A706368A360002B58DB042245
:10A7A000216891432160002854D1029D002B5AD08A
:10A7B0002500337842352B7055E05506DBD580B245
:10A7C000D9E71A680D68101D4969186013682E06CC
:10A7D00001D5196002E06D06FBD519800023029DAA
:10A7E00023614FE01A68111D196015680021626825
:10A7F000280000F0D5FC002801D0401B6060636891
:10A8000023610023029A13703CE023692A00049913
:10A810000398059DA847431C3ED023689B0715D489
:10A82000079BE068984239DA180037E022000123DC
:10A83000193204990398059EB047431C2CD001356A
:10A84000E368079A9B1AAB42F0DCE9E70025F7E7DB
:10A850000028ADD0029D3900FDF722FC735C013D5C
:10A860002B700028F7D1082F09D12368DB0706D504
:10A8700063682269934202DC3023013D2B70029B06
:10A880005B1B2361059B07AA00932100049B03988F
:10A89000FFF794FE431CB8D10120404209B0F0BD3F
:10A8A00021CE000032CE00000D4B70B51C680500B3
:10A8B000A36B002B0FD1182000F056FC094BA063AE
:10A8C0000360094B01224360084B83600B238381A3
:10A8D0000023026143610022A36B1D615A6170BDB8
:10A8E000640000200E33CDAB34126DE6ECDE0500C3
:10A8F000124B10B51C68A36B002B0FD1182000F071
:10A9000033FC0F4BA06303600E4B012243600E4BE0
:10A9100083600B238381002302614361A46B0B4A94
:10A92000206961690A4BFDF7F7FC012200238018BA
:10A930005941206161614800400810BD6400002059
:10A940000E33CDAB34126DE6ECDE05002D7F954C59
:10A950002DF451580CB430B5164B9DB00C1E1D682B
:10A9600008DA8B2301202B6040421DB030BC08BCAC
:10A9700002B01847822302A99B008B81002302901A
:10A9800008619C4200D0631E8B604B6101235B42D7
:10A99000CB81209A21AB2800019300F03DFD431CA0
:10A9A00001DA8B232B60002CDFD00023029A137076
:10A9B000DBE7C046640000200EB400B50B499CB034
:10A9C0001DAB02900690079104910948094904CBF8
:10A9D0000591006802A9019300F01EFD0023029A70
:10A9E00013701CB008BC03B01847C046FFFFFF7FC0
:10A9F000640000200802FFFF020010B51378541C09
:10AA0000002B05D1CC5CD4540133002CFAD110BDFD
:10AA10002200F3E702780B78002A03D001300131DD
:10AA20009A42F7D0D01A704703000A7801311A70A1
:10AA30000133002AF9D170470023C25C0133002A98
:10AA4000FBD1581E704730B50500002A00D130BD3B
:10AA50000C78013A6B1C2C700131002C05D19A182E
:10AA60009A42F4D01C700133FAE71D00EDE710B5EF
:10AA70000378002B0FD10B785A4253415B421840A8
:10AA800010BD0023CA5C002AFAD0C45C944201D1F4
:10AA90000133F7E701300378002BF2D11800EFE71C
:10AAA000F0B51F000E0087B00590019102920C983E
:10AAB000347800F0EAFA082200194378751C134034
:10AAC00036D12D2C36D1B51C74780126002F62D0DA
:10AAD000102F09D1302C07D120222B789343582BEB
:10AAE00054D110276C7802352D4B3900F31818001B
:10AAF0000393FDF7D5FA0491012100234942020096
:10AB00008C4618002100303909291AD80C00A742B8
:10AB100023DD591C09D06346824206D302D1049931
:10AB2000A14202DB0123784320182C780135E9E7A4
:10AB30002E00BCE72B2C01D01E00C7E7B51C747893
:10AB4000FAE721004139192901D8373CDFE7210014
:10AB50006139192901D8573CD9E75A1C08D1059AFF
:10AB600023331360029B0398002B09D107B0F0BD7B
:10AB7000002E00D04042029A002AF7D0002B01D0CC
:10AB80006B1E0193029B019A1A60EFE73024002F9D
:10AB9000AAD10827A8E7302C9ED00A27A4E7C046F0
:10ABA000FFFFFF7F37B51300064A05001068046AEF
:10ABB000002C00D1044C0A0000942900FFF770FF1C
:10ABC0003EBDC04664000020C8000020F8B5050066
:10ABD0000E001400002804D08369002B01D100F07E
:10ABE000C1F9224B9C422DD16C68A369A360A38953
:10ABF0001B0731D52369002B2ED023682269F7B2B9
:10AC0000981A6369F6B2834205DC2100280000F03F
:10AC10003BF9002826D1A3680130013BA3602368DB
:10AC20005A1C22601F706369834204D0A389DB072A
:10AC30001AD50A2E18D12100280000F025F9002885
:10AC400012D00FE00A4B9C4201D1AC68CDE7094B12
:10AC50009C42CAD1EC68C8E72100280000F00CF83B
:10AC60000028CAD0012676423000F8BD64CE00002C
:10AC700084CE000044CE0000364B70B51D6806003F
:10AC80000C00002D05D0AB69002B02D1280000F08C
:10AC900069F9314B9C420FD16C680C23E25E93B290
:10ACA00019072DD4D90611D4092301203360373375
:10ACB0001343A381404270BD284B9C4201D1AC6834
:10ACC000EBE7274B9C42E8D1EC68E6E75B0713D53E
:10ACD000616B002908D023004433994202D0300030
:10ACE00000F06AFA002363632422A3899343A381BB
:10ACF00000236360236923600823A2891343A3818F
:10AD00002369002B0BD1A0218022A3898900920006
:10AD10000B40934203D02100300000F0E1F9012301
:10AD2000A289134011D00023A36063695B42A36131
:10AD3000002023698342BED10C23E25E1306BAD5FC
:10AD400040231343A3810138B5E7920700D4636918
:10AD5000A360EDE76400002064CE000084CE000014
:10AD600044CE000010B5062000F090FC012000F059
:10AD7000CFFD0000F7B58A8905000C00130760D4E9
:10AD80004B68002B04DC0B6C002B01DC0020FEBDAB
:10AD9000E76A002FFAD000232E682B6080235B0126
:10ADA000216A1A4034D0606DA3895B0706D56368B9
:10ADB000C01A636B002B01D0236CC01A0200216AF9
:10ADC00000232800E76AB847A189431C06D12B68F5
:10ADD0001D2B30D82B4ADA40D3072CD500236360D3
:10ADE00023692360CB0405D5431C02D12B68002BBB
:10ADF00000D16065616B2E600029C7D02300443309
:10AE0000994202D0280000F0D7F900206063BEE725
:10AE100001232800B847431CC6D12B68002BC3D0A0
:10AE20001D2B01D0162B01D12E60AFE74023A28944
:10AE30001343A381ABE740230B430120A38140428E
:10AE4000A5E70F69002FA1D00B680F60DB1B0193F2
:10AE50000023920700D14B69A360019B002B00DC0B
:10AE600094E7019B3A00216A2800A66AB0470028AF
:10AE700003DC4023A2891343DFE7019B3F181B1A21
:10AE80000193EAE7010040200B6970B505000C0052
:10AE9000002B01D1002070BD002804D08369002B55
:10AEA00001D100F05FF80B4B9C4209D16C680C2279
:10AEB000A35E002BEED021002800FFF75BFFEAE73E
:10AEC000054B9C4201D1AC68F1E7044B9C42EED1AA
:10AED000EC68ECE764CE000084CE000044CE0000B5
:10AEE000002310B5040003604360836081814366E2
:10AEF000C281036143618361190008225C30FFF75E
:10AF000017FA054B24626362044BA362044BE362AD
:10AF1000044B236310BDC046CDB60000F5B600005B
:10AF20002DB7000059B7000010B5024900F08CF8A9
:10AF300010BDC04689AE000070B568254A1E554355
:10AF40000E002900743100F081F9041E08D00021A0
:10AF50002A00016046600C30A0606832FFF7E8F913
:10AF6000200070BD836913B50400002B28D18364D1
:10AF7000C3640365134B144A1B68826201939842B1
:10AF800001D101238361200000F020F860602000DF
:10AF900000F01CF8A060200000F018F80022E0602B
:10AFA00004216068FFF79CFF01220921A068FFF7D8
:10AFB00097FF02221221E068FFF792FF0123A361AD
:10AFC00013BDC0460CCE000029AF0000F8B51C4BE5
:10AFD00007001E68B369002B02D13000FFF7C2FFE3
:10AFE0004836B4687368013B04D53368002B07D03A
:10AFF0003668F6E70C22A55E002D0DD06834F2E726
:10B0000004213800FFF798FF30600028F0D10C23AE
:10B0100004003B602000F8BD20000A4B65662560F7
:10B020006560A560E36025616561A561082229006E
:10B030005C30FFF77DF96563A563A564E564E9E726
:10B040000CCE00000100FFFFF7B50400070000264A
:10B0500001914834002C01D13000FEBD6368A56821
:10B060000093009B013B009301D52468F2E7AB8974
:10B07000012B08D90E22AB5E013304D02900380021
:10B08000019B984706436835EBE7EC300068704752
:10B0900070B50E001D000E23C95E96B01400002985
:10B0A00007DA00232B60B3891B0611D48023DB0051
:10B0B0000FE06A4600F088FB0028F2DBF022019BDB
:10B0C00012021340054A9B185A4253412B60EDE788
:10B0D00040230020236016B070BDC04600E0FFFF93
:10B0E000F7B502268B8905000C00334206D02300F9
:10B0F00047332360236101236361F7BD01AB6A46D7
:10B10000FFF7C6FF00990700280000F09FF800280D
:10B1100008D10C22A35E9A05EFD4032293431E4369
:10B12000A681E4E70F4BAB628023A2892060134322
:10B13000A381009B20616361019B002B0DD00E2336
:10B14000E15E280000F052FB002806D00322A3890C
:10B1500093431A0001231343A381A0893843A0819C
:10B16000CBE7C04629AF000010B5034B01001868BB
:10B1700000F06CF810BDC0466400002082B00029C9
:10B1800000D101A9101E06D0002B06D013780B6049
:10B190001078431E984102B0704702204042FAE7FF
:10B1A000C9B28218904201D10020704703788B42C7
:10B1B000FBD00130F6E7000070B50500002910D083
:10B1C0000C1F2368002B00DAE418280000F034FB81
:10B1D0001D4A1368002B05D163601460280000F03D
:10B1E0002CFB70BDA34209D9216860188342F3D1BA
:10B1F00018685B6841182160EEE713005A68002A5E
:10B2000001D0A242F9D919685818A0420BD1206880
:10B210000918581819608242E0D110685268411824
:10B2200019605A60DAE7A04202D90C232B60D5E7F7
:10B2300021686018824203D1106852684118216069
:10B2400062605C60CAE7C046E01B0020032370B563
:10B25000CD1C9D43083506000C2D1ED20C25A9429D
:10B260001DD8300000F0E8FA254A146821000029B2
:10B2700019D1244C2368002B03D1300000F0CAF907
:10B2800020602900300000F0C5F9431C2BD10C23AD
:10B290003000336000F0D1FA03E0002DDFDA0C2338
:10B2A0003360002070BD0B685B1B19D40B2B03D9D6
:10B2B0000B60CC18256003E04B688C420DD1136005
:10B2C000300000F0BAFA200007220B30231D904313
:10B2D000C31AE7D05A42E250E4E763600C00EFE79C
:10B2E0000C004968C3E70323C41C9C43A042E1D07F
:10B2F000211A300000F08EF9431CDBD1C7E7C046AD
:10B30000E01B0020E41B0020F8B507000D0016002C
:10B31000002905D11100FFF799FF04002000F8BDB6
:10B32000002A03D1FFF748FF3400F7E700F086FA60
:10B330002C00B042F2D231003800FFF787FF041E24
:10B34000ECD029003200FEF7D7FF29003800FFF7C4
:10B3500033FFE3E7F0B58E6885B007000C00039279
:10B3600001939E423CD890238A89DB001A4234D054
:10B370000325096923685B1A0293636902985D4398
:10B38000EB0F5D19019B6D1001331B18AB4200D907
:10B390001D00530532D529003800FFF757FF061E60
:10B3A00009D10C233B6040230120A2894042134372
:10B3B000A38105B0F0BD029A2169FEF79DFFA38924
:10B3C000144A1A4080231343A381029B2661F61876
:10B3D00026606561019EED1AA560019B9E4200D921
:10B3E000019E320003992068FEF78FFFA3680020BA
:10B3F0009B1BA36023689E192660DAE72A003800A9
:10B40000FFF782FF061EE0D121693800FFF7D4FE66
:10B41000C7E7C0467FFBFFFFF0B59FB002900593E2
:10B420008B890F0016001B0611D50B69002B0ED15E
:10B430004021FFF70BFF38603861002805D10C234D
:10B44000029A013813601FB0F0BD40237B610023D6
:10B4500006AC6361203363761033A37635002B7816
:10B46000002B01D0252B46D1AB1B04930CD032000E
:10B4700039000298FFF76EFF431C00D1AEE062690D
:10B48000049B9446634463612B78002B00D1A5E0B4
:10B49000012200235242626002A9543252186E1CEB
:10B4A0002360E360A3601370A365317805225448DC
:10B4B000FFF776FE751C00281FD12268D30604D53D
:10B4C000532302A95B1820211970130704D55323B5
:10B4D00002A95B182B21197033782A2B16D035005E
:10B4E00000210A20E3682A786E1C303A092A4ED9D6
:10B4F000002918D010E00135B1E7414B2268C01A8D
:10B5000001238340134323602E00CEE7059B191DC2
:10B510001B680591002B01DB099304E05B42E360AB
:10B520000223134323602B782E2B0AD16B782A2B0E
:10B5300035D1059B02351A1D1B680592002B2BDBAC
:10B540000793304E297803223000FFF729FE0028A8
:10B5500006D04023801B83402268013513432360BB
:10B560002978062228486E1C2176FFF719FE00284C
:10B570003CD0264B002B25D10722059B0733934354
:10B58000083305936369039A9B18636166E7434335
:10B5900001219B183500A6E701235B42D0E7002379
:10B5A0000A201A000135636029786E1C3039092998
:10B5B00003D9002BC5D00792C3E742430123521899
:10B5C0003500F1E705AB00933A00114B21000298DA
:10B5D00000E000BF0390039B0133D3D1BB890B98DC
:10B5E0005B0600D42FE7012040422CE705AB009317
:10B5F0003A00074B21000298FFF74EF8EAE7C046F1
:10B6000010CE000016CE00001ACE00000000000090
:10B6100055B30000002370B5064C050008002360F8
:10B6200000F060F9431C03D12368002B00D02B608D
:10B6300070BDC046982F002070B504000D001F2972
:10B6400004D9162303600120404270BD436C002BD7
:10B6500004D08A009B181A68002A08D1200000F044
:10B6600031F82A000100200000F01AF8EDE7002070
:10B67000012AEAD0511C03D1162301302360E4E7EC
:10B68000002428001C6090472000DEE710B5034B23
:10B6900001001868FFF7D0FF10BDC046640000200D
:10B6A000002370B5064C050008001100236000F06F
:10B6B00001F9431C03D12368002B00D02B6070BD1F
:10B6C000982F002010B500F0E5F810BD70B50C0003
:10B6D0000E25495F00F0BAF8002803DB636D1B18E4
:10B6E000636570BDA389024A1340A381F9E7C04690
:10B6F000FFEFFFFFF8B51F008B8905000C00160057
:10B70000DB0505D50E23C95E0022022300F080F878
:10B71000A389054A28001340A38132000E23E15E6D
:10B720003B0000F02BF8F8BDFFEFFFFF70B50C00F9
:10B730000E25495F00F06CF8A389421C03D1054A2D
:10B740001340A38170BD802252011343A381606521
:10B75000F8E7C046FFEFFFFF10B50E23C95E00F00B
:10B7600021F810BD0B1E04D0FF2A04D98A230360E0
:10B770008B3B180070470A700123FAE770B505008B
:10B78000080011000022064C22601A0000F0B8F8F0
:10B79000431C03D12368002B00D02B6070BDC04632
:10B7A000982F0020002370B5064C05000800236088
:10B7B00000F060F8431C03D12368002B00D02B60FD
:10B7C00070BDC046982F0020002370B5064C0500C0
:10B7D00008001100236000F055F8431C03D12368D2
:10B7E000002B00D02B6070BD982F0020002370B577
:10B7F000064C05000800236000F054F8431C03D1F8
:10B800002368002B00D02B6070BDC046982F00200D
:10B8100070B50500080011000022064C22601A00D5
:10B8200000F050F8431C03D12368002B00D02B609C
:10B8300070BDC046982F0020704770470B1F1B68D3
:10B84000181F002B01DA0B58C018704770B505009F
:10B85000080011000022064C22601A0000F03AF89D
:10B86000431C03D12368002B00D02B6070BDC04661
:10B87000982F002058220120014B40421A60704747
:10B88000982F002058220120014B40421A60704737
:10B89000982F002058220120014B40421A60704727
:10B8A000982F00205822024B00201A607047C04693
:10B8B000982F002058220120014B40421A60704707
:10B8C000982F002058220120014B40421A607047F7
:10B8D000982F002058220120014B40421A607047E7
:10B8E000982F0020044A1368002B00D1034B18182E
:10B8F000106018007047C046E81B0020A02F0020F1
:10B9000058220120014B40421A607047982F0020B6
:10B91000FEE7C046F8B5C046F8BC08BC9E46704776
:10B92000F8B5C046F8BC08BC9E46704764617461B7
:10B9300000000000A8B90000EB010000B1B9000050
:10B9400017040000B9B900002D070000C0B90000BD
:10B950003D080000C5B90000DF020000D0B90000BA
:10B9600083040000D5B90000B5090000E1B900006A
:10B970001B020000EBB9000035060000F9B9000019
:10B98000A105000072616E646F6D00616C6C006CEB
:10B990006173740066616C7365007472756500256F
:10B9A0002E3135732E2E2E006D616B654C697374CC
:10B9B000006164644C6173740064656C6574650057
:10B9C0006A6F696E00636F707946726F6D546F00B5
:10B9D00066696E64006A6F696E537472696E67732C
:10B9E00000756E69636F6465417400756E69636F9D
:10B9F0006465537472696E6700667265654D656D46
:10BA00006F727900C80F0000D80F0000F20F00001D
:10BA100070100000A8100000DE10000016110000D9
:10BA20003C11000078110000BA1100001012000053
:10BA300054120000C0120000081300002E13000072
:10BA400066130000AC130000D213000000140000C5
:10BA5000321400006A140000EE140000B615000055
:10BA60002C16000098160000E016000000170000D9
:10BA700022170000D217000018180000C80F00009D
:10BA8000C80F0000C80F000090180000F818000050
:10BA900060190000C0190000081A00007A1A00009E
:10BAA000EC1A0000341B00007A1B0000B01B0000E1
:10BAB000F61B00003C1C0000841C0000D81C000089
:10BAC0002C1D0000741D0000DE1D0000141E00006F
:10BAD0005C1E0000A41E0000EC1E0000261F0000DB
:10BAE0006E1F0000B61F0000C80F0000C80F000046
:10BAF000C80F00001E200000C80F000054200000E6
:10BB000080200000B6200000E2200000C80F0000E6
:10BB1000C80F0000C80F0000C80F00001821000067
:10BB20005A210000C80F0000C80F0000AA21000021
:10BB3000FA21000020220000C80F0000C80F0000FA
:10BB4000C80F00004E2200007E220000AE2200003E
:10BB5000E42200000E230000442300006E230000B6
:10BB600096230000BE230000EE2300001E240000E8
:10BB70004824000072240000A2240000CC2400000D
:10BB8000C80F0000C80F0000C80F0000C80F000059
:10BB9000C80F0000FC240000282500006C250000D0
:10BBA00098250000C4250000FA250000302600007A
:10BBB000662600009C260000C8260000F42600002F
:10BBC0002A270000C80F0000C80F0000C80F00009F
:10BBD000C80F0000C80F0000C80F0000C80F000009
:10BBE000C80F0000C80F0000C80F0000C80F0000F9
:10BBF000C80F0000C80F0000C80F00005627000043
:10BC00008C270000282564206974656D206C697399
:10BC1000742900286F626A65637420747970653ACC
:10BC20002025642900537461636B20756E6465720E
:10BC3000666C6F7700000000070000000300000042
:10BC400081BC00007128000089BC0000752800003C
:10BC500092BC00006D2800009BBC00007928000009
:10BC600015000000010000000200000004000000B8
:10BC7000050000000600000043616C6C696F706590
:10BC800000686173546F6E6500706C6179546F6EFB
:10BC90006500686173536572766F007365745365F0
:10BCA00072766F00474320746F6F6B202564207598
:10BCB000736563733B206672656520256420776F2A
:10BCC000726473003C496E74656765723E003C4F58
:10BCD000626A6563743E003C4C6973743E000D0AF1
:10BCE000564D2050616E69633A2025730D0A006D30
:10BCF0006973630004BD0000193100000DBD000030
:10BD0000D1300000686578546F496E740073696EB5
:10BD10000000000060BD00008531000068BD00002B
:10BD20008931000072BD0000A73100007BBD00001A
:10BD3000B131000086BD0000BB31000092BD0000A3
:10BD4000C5310000A3BD0000CF310000B9BD000027
:10BD500093310000D2BD00009D3100006E6574007B
:10BD600068617357694669007374617274576946F4
:10BD7000690073746F705769466900776966695323
:10BD80007461747573006D794950416464726573B0
:10BD900073007468696E674465736372697074696F
:10BDA0006F6E00636C6561725468696E6744657399
:10BDB0006372697074696F6E00617070656E64544F
:10BDC0006F5468696E674465736372697074696FF4
:10BDD0006E00617070656E64546F5468696E675070
:10BDE000726F7065727479000D0E0F04050C0B0AEA
:10BDF0000607080904050C0B0A06070809000000DD
:10BE0000000008080800080A4A4000000A5FEA5FCC
:10BE1000EA0ED92ED36E19324489330C924C924DCE
:10BE200008080000000488080804080484848800C6
:10BE30000A448A4000048EC4800000000488000088
:10BE40000EC000000000080001224488100C92522D
:10BE5000524C048C84848E1C824C901E1EC24492D0
:10BE60004C06CA525FE21FF01EC13E02448ED12E24
:10BE70001FE24488100ED12ED12E0ED12EC4880080
:10BE80000800080000048004880244880482000E30
:10BE9000C00EC008048244880ED126C0040ED135DD
:10BEA000B36C0C925ED2521C925C925C0ED010105D
:10BEB0000E1C9252525C1ED01C901E1ED01C901064
:10BEC0000ED013712E12525ED2521C8808081C1F0D
:10BED000E242524C1254981492101010101E113B52
:10BEE00075B131113935B3710C9252524C1C925CC0
:10BEF00090100C92524C861C925C92510ED00C8287
:10BF00005C1FE4848484125252524C1131312A4411
:10BF1000113135BB7112524C9252112A4484841E45
:10BF2000C488101E0EC808080E10080482410EC2F4
:10BF300042424E048A400000000000001F080480B6
:10BF40000000000ED2524F10101C925C000ED01058
:10BF50000E02424ED24E0C925C900E06C81C88080F
:10BF60000ED24EC24C10101C925208000808080253
:10BF70004002424C10149814920808080806001B4E
:10BF800075B131001C925252000C92524C001C921E
:10BF90005C90000ED24EC2000ED010100006C804F5
:10BFA0009808080EC807001252524F0011312A4457
:10BFB00000113135BB00124C8C9200112A449800BC
:10BFC0001EC4881E06C48C84860808080808180841
:10BFD0000C881800000C83600000000001000000C5
:10BFE0000200000003000000040000000500000043
:10BFF0000600000007000000080000000900000023
:10C000000A0000000B0000000C0000000D00000002
:10C010000E0000000F0000001000000012000000E1
:10C020001400000016000000180000001A000000B4
:10C030001C0000001E000000200000002300000083
:10C0400026000000290000002C0000002F00000046
:10C0500032000000360000003A0000003E00000000
:10C0600042000000460000004B00000050000000AD
:10C07000550000005A000000610000006800000048
:10C080006F000000760000007D00000084000000CA
:10C090008B0000009200000099000000A00000004A
:10C0A000A7000000AE000000B5000000BC000000CA
:10C0B000C3000000CA000000D1000000D80000004A
:10C0C000DF000000E6000000ED000000F4000000CA
:10C0D000FB000000FF00000028C10000F531000057
:10C0E00033C10000293700003DC100003934000091
:10C0F0004AC100005934000051C10000A9340000B9
:10C100005AC10000F934000066C10000D5330000B8
:10C1100077C100003936000084C10000F536000008
:10C12000646973706C6179006C696768744C6576DA
:10C13000656C006D62446973706C6179006D624476
:10C140006973706C61794F6666006D62506C6F74D4
:10C15000006D62556E706C6F74006D624472617731
:10C160005368617065006D625368617065466F72F7
:10C170004C6574746572006E656F506978656C53B8
:10C18000656E64006E656F506978656C53657450B8
:10C19000696E004E6F7420656E6F75676820726FF0
:10C1A0006F6D206576656E20616674657220636FC1
:10C1B0006D70616374696F6E00436F6D706163745D
:10C1C000656420466C61736820636F6465207374D6
:10C1D0006F72650A256420627974657320757365D2
:10C1E0006420282564252529206F662025640042C7
:10C1F0006164207265636F726420666F756E64207F
:10C20000647572696E6720696E697469616C697AB8
:10C210006174696F6E0025642025642025642028E0
:10C22000256420776F72647329002564207265632A
:10C230006F7264732C20256420776F7264732C20D6
:10C240006D617849442025642C20636F6D706163B3
:10C2500074696F6E206379636C6573202564005286
:10C260006573746F726564202564207363726970EE
:10C270007473005374617274656400726164696FF1
:10C280000000000012C30000F94000001FC30000BE
:10C29000694300002FC30000094300003DC30000B4
:10C2A000E944000048C300001141000058C30000E9
:10C2B000854100006CC30000214100007BC30000E9
:10C2C000CB46000087C300004946000090C3000031
:10C2D000ED4500009BC3000035450000A6C30000EB
:10C2E00071450000AFC30000A5450000B8C30000C1
:10C2F000354100006E756D626572006E6F6E65008F
:10C300006F74686572007061697200737472696E2F
:10C31000670064697361626C65526164696F006D86
:10C3200065737361676552656365697665640070FE
:10C3300061636B65745265636569766500706163FE
:10C340006B657453656E64007265636569766564D8
:10C35000496E7465676572007265636569766564C8
:10C360004D657373616765547970650072656365C7
:10C3700069766564537472696E670073656E6449AB
:10C380006E74656765720073656E645061697200F2
:10C3900073656E64537472696E6700736574436885
:10C3A000616E6E656C0073657447726F75700073B3
:10C3B0006574506F776572007369676E616C537452
:10C3C00072656E67746800000000000096300777A1
:10C3D0002C610EEEBA51099919C46D078FF46A7079
:10C3E00035A563E9A395649E3288DB0EA4B8DC7999
:10C3F0001EE9D5E088D9D2972B4CB609BD7CB17E19
:10C40000072DB8E7911DBF906410B71DF220B06AE8
:10C410004871B9F3DE41BE847DD4DA1AEBE4DD6DF8
:10C4200051B5D4F4C785D38356986C13C0A86B64F8
:10C430007AF962FDECC9658A4F5C0114D96C066318
:10C44000633D0FFAF50D088DC8206E3B5E10694CF8
:10C45000E44160D5727167A2D1E4033C47D4044B38
:10C46000FD850DD26BB50AA5FAA8B5356C98B24218
:10C47000D6C9BBDB40F9BCACE36CD832755CDF4598
:10C48000CF0DD6DC593DD1ABAC30D9263A00DE51C8
:10C490008051D7C81661D0BFB5F4B42123C4B356B8
:10C4A0009995BACF0FA5BDB89EB802280888055F38
:10C4B000B2D90CC624E90BB1877C6F2F114C685898
:10C4C000AB1D61C13D2D66B69041DC760671DB0186
:10C4D000BC20D2982A10D5EF8985B1711FB5B60658
:10C4E000A5E4BF9F33D4B8E8A2C9077834F9000F98
:10C4F0008EA8099618980EE1BB0D6A7F2D3D6D0838
:10C50000976C6491015C63E6F4516B6B62616C1C27
:10C51000D83065854E0062F2ED95066C7BA5011B57
:10C52000C1F4088257C40FF5C6D9B06550E9B712F7
:10C53000EAB8BE8B7C88B9FCDF1DDD62492DDA15B7
:10C54000F37CD38C654CD4FB5861B24DCE51B53AD7
:10C550007400BCA3E230BBD441A5DF4AD795D83DD7
:10C560006DC4D1A4FBF4D6D36AE96943FCD96E3417
:10C57000468867ADD0B860DA732D0444E51D0333F7
:10C580005F4C0AAAC97C0DDD3C710550AA41022707
:10C5900010100BBE86200CC925B56857B3856F20D7
:10C5A00009D466B99FE461CE0EF9DE5E98C9D92937
:10C5B0002298D0B0B4A8D7C7173DB359810DB42E77
:10C5C0003B5CBDB7AD6CBAC02083B8EDB6B3BF9AC3
:10C5D0000CE2B6039AD2B1743947D5EAAF77D29D4F
:10C5E0001526DB048316DC73120B63E3843B64942F
:10C5F0003E6A6D0DA85A6A7A0BCF0EE49DFF09932F
:10C6000027AE000AB19E077D44930FF0D2A308879E
:10C6100068F2011EFEC206695D5762F7CB6765804E
:10C6200071366C19E7066B6E761BD4FEE02BD3894E
:10C630005A7ADA10CC4ADD676FDFB9F9F9EFBE8EAE
:10C6400043BEB717D58EB060E8A3D6D67E93D1A1EE
:10C65000C4C2D83852F2DF4FF167BBD16757BCA6CE
:10C66000DD06B53F4B36B248DA2B0DD84C1B0AAF6E
:10C67000F64A0336607A0441C3EF60DF55DF67A8EE
:10C68000EF8E6E3179BE69468CB361CB1A8366BC7E
:10C69000A0D26F2536E2685295770CCC03470BBBCE
:10C6A000B91602222F260555BE3BBAC5280BBDB2CE
:10C6B000925AB42B046AB35CA7FFD7C231CFD0B56E
:10C6C0008B9ED92C1DAEDE5BB0C2649B26F263EC60
:10C6D0009CA36A750A936D02A906099C3F360EEB6E
:10C6E0008567077213570005824ABF95147AB8E22E
:10C6F000AE2BB17B381BB60C9B8ED2920DBED5E50E
:10C70000B7EFDC7C21DFDB0BD4D2D38642E2D4F15D
:10C71000F8B3DD686E83DA1FCD16BE815B26B9F6ED
:10C72000E177B06F7747B718E65A0888706A0FFF4D
:10C73000CA3B06665C0B0111FF9E658F69AE62F80D
:10C74000D3FF6B6145CF6C1678E20AA0EED20DD70D
:10C750005483044EC2B30339612667A7F71660D02D
:10C760004D476949DB776E3E4A6AD1AEDC5AD6D96D
:10C77000660BDF40F03BD83753AEBCA9C59EBBDE8D
:10C780007FCFB247E9FFB5301CF2BDBD8AC2BACA3D
:10C790003093B353A6A3B4240536D0BA9306D7CDAD
:10C7A0002957DE54BF67D9232E7A66B3B84A61C4CD
:10C7B000021B685D942B6F2A37BE0BB4A18E0CC38D
:10C7C0001BDF055A8DEF022D416C6C207461736B79
:10C7D000732073746F70706564007630373000209A
:10C7E0002573202573004D656D6F727920636C652C
:10C7F00061726564004E6F206672656520746173B6
:10C800006B20656E747269657300000054C8000087
:10C810006558000061C80000CB5800006DC80000DA
:10C820009B58000073C80000AB58000079C8000096
:10C83000BB5800007FC800009955000089C800005F
:10C84000E958000091C80000C556000073656E737A
:10C850006F727300616363656C65726174696F6E9A
:10C860000074656D70657261747572650074696CD1
:10C8700074580074696C74590074696C745A00744B
:10C880006F75636852656164006932635265616403
:10C8900000693263577269746500000010C90000B6
:10C8A000695900001EC900006D59000027C9000029
:10C8B0007959000031C900007D5900003AC90000D3
:10C8C000815900003FC900008559000044C900009B
:10C8D0008959000050C900008D59000057C9000057
:10C8E0009159000060C900009559000065C9000019
:10C8F0009959000070C900009D5900007AC90000D4
:10C900007159000084C900007559000074667400F4
:10C91000656E61626C65446973706C61790067650E
:10C9200074576964746800676574486569676874FA
:10C9300000736574506978656C006C696E6500728F
:10C9400065637400726F756E64656452656374002C
:10C95000636972636C6500747269616E676C65000F
:10C960007465787400746674546F756368656400E8
:10C97000746674546F7563685800746674546F7588
:10C9800063685900746674546F7563685072657398
:10C99000737572650057656C636F6D6520746F20E9
:10C9A0004D6963726F426C6F636B732100705F73CC
:10C9B000706920213D204E554C4C002F686F6D65ED
:10C9C0002F62726F6D61676F73612F2E706C61746F
:10C9D000666F726D696F2F7061636B616765732F2E
:10C9E0006672616D65776F726B2D61726475696EC9
:10C9F0006F6E6F726469636E7266352F6C696272F6
:10CA000061726965732F5350492F5350492E6370DB
:10CA10007000535049436C6173733A3A5350494321
:10CA20006C617373284E52465F5350495F5479705E
:10CA3000652A2C2075696E74385F742C2075696EB8
:10CA400074385F742C2075696E74385F7429000027
:10CA50000000000000000000A15B00005D5B000022
:10CA6000835B00008D5B0000975B0000815B000032
:10CA7000000000000100000002000000160000009D
:10CA80000400000005000000060000000700000090
:10CA900008000000090000000A0000000B00000070
:10CAA0000C0000000D0000000E0000000F00000050
:10CAB0001A0000001B00000014000000130000001A
:10CAC0001100000003000000100000001C00000026
:10CAD0001D0000001E0000001200000015000000F4
:10CAE00017000000180000001900000000000000FE
:10CAF000000000005160000081670000D16000006C
:10CB0000E5600000DB6000004D6000004160000057
:10CB1000F16000006D6000003D600000000000005A
:10CB2000000000000000304300000000000030C39F
:10CB30007371727400000000FB21F93FFB21094072
:10CB40007CD91240FB2119407A6A1F407CD92240CF
:10CB5000BBFD2540FB2129403A462C407A6A2F40F4
:10CB60005C4731407CD932409C6B3440BBFD354042
:10CB7000DB8F3740FB2139401BB43A403A463C40FA
:10CB80005AD83D407A6A3F404C7E40405C47414025
:10CB90006C1042407CD942408CA243409C6B444084
:10CBA000AC344540BBFD4540CBC64640DB8F4740DB
:10CBB000EB584840FB21494083F9A200444E6E00E7
:10CBC000FC291500D1572700DD34F50062DBC000D9
:10CBD0003C999500419043006351FE00BBDEAB00E1
:10CBE000B761C5003A6E2400D24D42004906E0000C
:10CBF00009EA2E001C92D100EB1DFE0029B11C0099
:10CC0000E83EA700F535820044BB2E009CE9840075
:10CC1000B4267000417E5F00D691390053833900FD
:10CC20009CF439008B5F840028F9BD00F81F3B009D
:10CC3000DEFF97000F980500112FEF000A5A8B00B6
:10CC40006D1F6D00CF7E360009CB2700464FB70021
:10CC50009E663F002DEA5F00BA277500E5EBC7002E
:10CC60003D7BF100F739070092528A00FB6BEA0026
:10CC70001FB15F00085D8D00300356007BFC46004D
:10CC8000F0AB6B0020BCCF0036F49A00E3A91D0086
:10CC90005E619100081BE60085996500A0145F00A5
:10CCA0008D40680080D8FF0027734D0006063100D4
:10CCB000CA561500C9A873007BE260006B8CC000E7
:10CCC00000000040FB21F93F000000002D44743EAD
:10CCD000000000809846F83C0000006051CC783B92
:10CCE00000000080831BF0390000004020257A38C6
:10CCF000000000802282E336000000001DF3693549
:10CD00000200000003000000040000000600000014
:10CD1000648400000E8400000E8400003C85000046
:10CD20000A8400000A840000328500003C8500006F
:10CD30000A840000328500000A8400003C8500005F
:10CD400040850000408500004085000048850000C7
:10CD5000408F0000B28D0000F68D00005A8D00005B
:10CD6000F68D0000E68E0000F68D00005A8D000062
:10CD7000B28D0000B28D0000E68E00005A8D0000DA
:10CD8000528D0000528D0000528D0000F48E000084
:10CD9000689600006A9500006A9500008898000077
:10CDA0006495000064950000709800008898000069
:10CDB0006495000070980000649500008898000059
:10CDC0007E9800007E9800007E9800008C980000FD
:10CDD0002C2066756E6374696F6E3A200061737300
:10CDE000657274696F6E2022257322206661696CFA
:10CDF00065643A2066696C6520222573222C206CBC
:10CE0000696E65202564257325730A00680000207B
:10CE1000232D302B2000686C4C0065666745464723
:10CE200000303132333435363738394142434445A6
:10CE30004600303132333435363738396162636415
:10CE40006566000000000000000000000000000017
:10CE500000000000000000000000000000000000D2
:10CE600000000000000000000000000000000000C2
:10CE700000000000000000000000000000000000B2
:10CE800000000000000000000000000000000000A2
:10CE90000000000000000000000000000000000092
:10CEA000000000004300504F53495800002020204C
:10CEB000202020202020282828282820202020204A
:10CEC000202020202020202020202020208810101A
:10CED0001010101010101010101010101004040476
:10CEE0000404040404040410101010101010414134
:10CEF0004141414101010101010101010101010122
:10CF00000101010101010101101010101010424235
:10CF100042424242020202020202020202020202F1
:10CF20000202020202020202101010102000000091
:10CF300000000000000000000000000000000000F1
:10CF400000000000000000000000000000000000E1
:10CF500000000000000000000000000000000000D1
:10CF600000000000000000000000000000000000C1
:10CF700000000000000000000000000000000000B1
:10CF800000000000000000000000000000000000A1
:10CF90000000000000000000000000000000000091
:10CFA0000000000000000000000000000000000081
:04CFB000000000007D
:08CFB4005431FF7F0100000071
:10CFBC00FFFFFFFF400600001800000019FCFFFFF8
:10CFCC00FFFFFFFF0200000003000000FFFFFFFF58
:10CFDC000000000001000000000002000100000041
:10CFEC00FFFFFFFF00000000020000000000040033
:10CFFC0002000000FFFFFFFF000000000300000024
:10D00C0000000800030000000A00000008000000F7
:10D01C0001000000680000200000000064CE000049
:10D02C0084CE000044CE0000000000000000000090
:10D03C0000000000000000000000000000000000E4
:10D04C0000000000000000000000000000000000D4
:10D05C0000000000000000000000000000000000C4
:10D06C0000000000000000000000000000000000B4
:10D07C000000000000000000430000000000000061
:10D08C000000000000000000000000000000000094
:10D09C000000000000000000430000000000000041
:10D0AC000000000000000000000000000000000074
:10D0BC000000000000000000430000000000000021
:10D0CC000000000000000000000000000000000054
:10D0DC000000000000000000430000000000000001
:10D0EC000000000000000000000000000000000034
:10D0FC0000000000000000004300000000000000E1
:10D10C000000000000000000000000000000000013
:10D11C0000000000000000004300000000000000C0
:10D12C0000000000000000000000000000000000F3
:10D13C0000000000000000004300000000000000A0
:10D14C0000000000000000000000000000000000D3
:10D15C00000000000000000065B700007DB1000079
:10D16C0000000000ACCE0000A6B90000EEBC000030
:10D17C00EEBC0000EEBC0000EEBC0000EEBC0000FB
:10D18C00EEBC0000EEBC0000EEBC0000EEBC0000EB
:10D19C00FFFFFFFFFFFFFFFFFFFFFFFFFFFF000091
:10D1AC000100415343494900000000000000000009
:10D1BC000000000000000000000000000000000063
:10D1CC0000004153434949000000000000000000EA
:10D1DC000000000000000000000000000000000043
:10D1EC0000000000E90000002D5B0000755E0000EF
:08D1FC009D630000C10000006A
:0400000300005F1189
:00000001FF
